:1000000016C3000033C3000031C300002FC300003B
:100010002DC300002BC3000029C3000027C300002C
:1000200025C3000023C3000021C300001FC300003C
:100030000C94583C1BC3000019C3000017C30000F8
:1000400015C3000013C300000C94443C0FC3000010
:100050000DC300000BC3000009C3000007C300006C
:1000600005C3000003C3000001C30000FFC200007D
:10007000FDC20000FBC20000F9C20000F7C2000090
:10008000F5C20000F3C20000F1C20000180A1D0A08
:100090002B0A300A350A3A0A3F0A440AD20DD70D14
:1000A000E50DEA0DEF0DF40DF90DFE0D38123B12C2
:1000B0003E124112441247124A124D12C81DED1D44
:1000C000011E141E171E281E391E571EDE1DE11D9F
:1000D0004A1E4D1E501EE41DE71DEA1D54236A23CF
:1000E0007E239623AC23C223E623FC231224DC25A3
:1000F000332629278027762878293A2A0C2B0D2C9D
:10010000482C9C2CDD2CE62C362D862D892D8C2D13
:100110008F2D922D952D982D9B2D45305B30713074
:1001200088309E30B430CA30E030343137313A3123
:100130003D314031433146314931A1311D3299328F
:100140002233AB3322349E341A3596350F367C3643
:10015000F3367937FC37000000000000000004048B
:100160000404000400000A0A0A00000000000A0A51
:100170001F0A1F0A0A00040F140E051E0400181996
:100180000204081303000C12140814120D000C04CE
:100190000800000000000204080808040200080427
:1001A0000202020408000004150E150400000004F9
:1001B000041F04040000000000000C0408000000FC
:1001C000001F0000000000000000000C0C000001F7
:1001D0000204081000000E11131519110E00040C72
:1001E000040404040E000E11010204081F001F0283
:1001F000040201110E0002060A121F0202001F1063
:100200001E0101110E000608101E11110E001F0123
:100210000204080808000E11110E11110E000E1133
:10022000110F01020C000001020408100000000C74
:100230000C000C040800020408100804020000006E
:100240001F001F00000008040201020408000E1134
:100250000102040004000E11010D15150E000E110F
:1002600011111F1111001E11111E11111E000E116E
:10027000101010110E001C12111111121C001F1071
:10028000101E10101F001F10101E101010000E1155
:10029000101711110E001111111F111111000E0470
:1002A000040404040E000702020202120C001112E0
:1002B0001418141211001010101010101F00111B30
:1002C00015151111110011111915131111000E112D
:1002D000111111110E001E11111E101010000E111F
:1002E000111115120D001E11111E141211000F1004
:1002F000100E01011E001F04040404040400111167
:10030000111111110E0011111111110A0400111116
:10031000111115150E0011110A040A111100111105
:10032000110A040404001F01020408101F000E0833
:10033000080808080E00110A1F041F0404000E021A
:10034000020202020E00040A110000000000000078
:10035000000000001F000804000000000000000072
:100360000E010F110F0010101E1111111E000000C0
:100370000E1010110E0001010D1311110F000000DD
:100380000E111F100E000609081C08080800000FB7
:1003900011110F010E001010161911111100040097
:1003A0000C0404040E000200060202120C001010DD
:1003B0001214181412001808080808081C0000007D
:1003C0001A15151111000000161911111100000065
:1003D0000E1111110E0000001E111E101000000061
:1003E0000F110F010100000016191010100000007D
:1003F0000E100E011E0008081C0808090600000067
:10040000111111130D0000001111110A0400000058
:10041000111111150A000000110A040A1100000050
:1004200011110F010E0000001F0204081F003844C4
:1004300044447C4444007C40407844447800784400
:100440004478444478007C404040404040000C14D4
:10045000242424243C447C40407840407C00545474
:100460005438545454003844041804443800444464
:100470004C546444440054444C5464444400444840
:100480005060504844001C24242424246400446CFC
:100490005454444444004444447C44444400384458
:1004A0004444444438007C44444444444400784434
:1004B00044784040400038444040404438007C107C
:1004C0001010101010004444443C044438003854C8
:1004D0005454381010004444281028444400444424
:1004E000444444447E02444444443C040400545480
:1004F000545454547C005454545454547E02602038
:100500002038242438004444446454546400404057
:100510004078444478003844041C0444380048546B
:100520005474545448003C44443C14244400000097
:1005300038043C443C0000007840784478000000D7
:10054000784C784C78000000784040404000000033
:10055000182828287C44000038447C403C000000D7
:1005600054543854540000007804380478000000D3
:10057000444C546444000010444C54644400000053
:1005800044487048440000001C24444444000000D7
:10059000446C545444000000484878484800000027
:1005A0003844444438000000784848484800000077
:1005B0007048704040000000384040403800000063
:1005C0007C1010101000000048483808700000002F
:1005D000385454381000000044281028440000000B
:1005E000484848487C040000484838080800000093
:1005F000545454547C000000545454547E0200005F
:1006000060203C223C0000004242724A720000001E
:1006100040407844780000007008780870000000BE
:100620004C5272524C0000003C443C4444001124A3
:100630001FBECFEFD0E1DEBFCDBF15E0A0E0B1E03F
:10064000E4EEF4E800E00BBF02C007900D92A63D77
:10065000B107D9F726E0A6EDB5E001C01D92A83894
:10066000B207E1F70E94B63C0C947042C9CCE2E6B6
:10067000F0E090819E7F9083908194609083908140
:10068000977F9083A8988BBB8DE08A95F1F7000047
:10069000A89A8081886080830895E2E6F0E09081E6
:1006A000916090839081946090839081977F9083F4
:1006B000A8988BBB8DE08A95F1F70000A89A8081FD
:1006C000886080830895CF93C82F892FE6DF8C2F11
:1006D000CF91E3CFE2E6F0E020812160208320810A
:1006E000246020832081277F2083A8988BBB92BB26
:1006F0008DE08A95F1F70000A89A80818860808358
:100700000895CF93C82F86E3B2DFC13049F030F0AF
:10071000C23041F0C33059F488EE07C088E403C00A
:1007200088E203C088E8B9DF04C0B7DF0BC0CD7F23
:1007300049F48FEE90E09093D9058093D8058FE32C
:1007400091E008C08FE391E09093D9058093D8059C
:100750008FEE90E09093D7058093D605CF910895C2
:10076000CF93C82F8FEF8ABB81BB8093610081E05C
:1007700084BBE2E6F0E080818260808381E077DF05
:100780002FEF89E698E1215080409040E1F700C0CA
:10079000000080EC6CDF85E280DF81EC68DF81E1C6
:1007A0007CDF85EC64DF8BE278DF8BE276DF87EC41
:1007B0005EDF86E872DF8C2FA4DF8AE358DF85E0F6
:1007C0006CDF81EB54DF80E068DF88E166DF86EB79
:1007D0004EDF8AE062DF82E860DF87E25EDF81E190
:1007E00046DF2FEF8DEE92E0215080409040E1F700
:1007F00000C0000089E2CF913ACF0F931F93CF93AF
:10080000DF938C01EB018AE232DFC8015CDFCE01AD
:10081000DF91CF911F910F9156CF0F931F93CF93DD
:10082000DF938C01EB018BE222DFC8014CDFCE01AC
:10083000DF91CF911F910F9146CFCF93DF93EB01C3
:10084000BC01DBDFBE01CE01E8DF8CE2DF91CF919E
:100850000ECFCF93DF93EA01F0DFCE01DF91CF918E
:1008600039CF8F929F92AF92BF92CF92DF92EF9249
:10087000FF920F931F93CF93DF93A8956817790783
:1008800038F4862797276827792786279727A895FA
:100890002417350738F442275327242735274227C2
:1008A0005327A895A091D805B091D905FC01A817A8
:1008B000B90708F4FD016B01A617B70708F46D012D
:1008C0008091D6059091D705EA018417950708F421
:1008D000EC0179018217930708F47C01A895960131
:1008E0002F5F3F4F2E1B3F0BD7011196AC1BBD0B4B
:1008F0000E94383F4B015C01B601CF017EDFA89515
:10090000B701CE018ADF8CE2B2DEA895C12CD12CD2
:100910007601C814D904EA04FB0449F0C801DADE00
:10092000A8958FEFC81AD80AE80AF80AF2CFDF9123
:10093000CF911F910F91FF90EF90DF90CF90BF90DC
:10094000AF909F908F9008950F931F93411551057D
:1009500079F02115310561F0FA01AB01615071099F
:10096000260F371FBC01615071096E0F7F1F79DFA1
:100970001F910F9108952F923F924F925F926F9225
:100980007F928F929F92AF92BF92CF92DF92EF921F
:10099000FF920F931F93CF93DF93CDB7DEB7679787
:1009A0000FB6F894DEBF0FBECDBF5C01798B688BAC
:1009B000598748873B872A870F83F12C28E0029FBD
:1009C000C00111241A821982E8E0F0E0FF8BEE8B5F
:1009D00047019C01285F31093B8B2A8BFC01E052C7
:1009E000F340FD8BEC8BC888D98889819A81C80E29
:1009F000D91E8A899B89EE89FF898E1B9F0B9C01DA
:100A00002A5A3E4F3F872E878C899D898E1B9F0BCC
:100A1000FC01EA5AFE4FFD87EC871E821D821C8274
:100A20001B8287E0682E712C412C512C212C312CFB
:100A3000FF81F7FD1EC0EE85FF85849190E0062CB6
:100A400002C0959587950A94E2F780FF08C0088553
:100A500019859701A701B6018D819E8107C00A857E
:100A60001B859701A701B6018B819C818A0D9B1D77
:100A700020C0FF81F03CF0F0EC85FD85849190E092
:100A8000062C02C0959587950A94E2F780FF09C06D
:100A9000088519859701A701B601C501820D931D2F
:100AA00008C00A851B859701A701B601C501840D01
:100AB000951D4ADF280C391C480C591CF1E06F1AAF
:100AC00071082B813C81280D391D3C832B838D813E
:100AD0009E81880D991D9E838D839FEF69167906EF
:100AE00009F0A6CFEE89FF893197FF8BEE8B298124
:100AF0003A812E0D3F1D3A832983EF2B09F073CFE6
:100B000067960FB6F894DEBF0FBECDBFDF91CF91D1
:100B10001F910F91FF90EF90DF90CF90BF90AF901B
:100B20009F908F907F906F905F904F903F902F900D
:100B300008954F925F926F927F928F929F92AF92A1
:100B4000BF92CF92DF92EF92FF920F931F93CF93BA
:100B5000DF93EC016B014A013901102F88E0089FF7
:100B6000500111242701F20101912F010023B1F05E
:100B70002091D8053091D905CE010896281739075C
:100B800020F4CA0CDB1CC1E0D0E0E12E9301A401EB
:100B9000B601CE01F0DECA0DDB1DE5CFDF91CF91AE
:100BA0001F910F91FF90EF90DF90CF90BF90AF908B
:100BB0009F908F907F906F905F904F9008956F926D
:100BC0007F928F929F92AF92BF92CF92DF92EF92DD
:100BD000FF920F93CF93DF9300D000D0CDB7DEB755
:100BE0006C015B014A013901C70119821A821B821B
:100BF0001C824AE0BE016F5F7F4F0E94473FCE01DB
:100C000001967C019301A401B501C60192DF0F900A
:100C10000F900F900F90DF91CF910F91FF90EF9079
:100C2000DF90CF90BF90AF909F908F907F906F900C
:100C300008950F931F932091D6053091D7056091A9
:100C4000D8057091D9058C0140E050E080E090E03B
:100C500008DE1F910F910895EF92FF920F931F935B
:100C6000CF93DF93EB018A017901BC01640F751FFB
:100C7000C4DDBE01CE01D1DD8CE2F9DCC0E0D0E004
:100C8000C017D10721F0C70125DD2196F9CFDF91EB
:100C9000CF911F910F91FF90EF900895EF92FF92E7
:100CA0000F931F93CF93DF93EB018A017901BC016E
:100CB000A4DDBE01600F711FCE01AFDD8CE2D7DC79
:100CC000C0E0D0E0C017D10721F0C70103DD2196B5
:100CD000F9CFDF91CF911F910F91FF90EF90089581
:100CE0002F923F924F925F926F927F928F929F923C
:100CF000AF92BF92CF92DF92EF92FF920F931F932A
:100D0000CF93DF9300D000D000D0CDB7DEB76C0119
:100D10007B015A0139012801261B370B3A832983AD
:100D20008A01081B190B17FF03C0119501951109C2
:100D3000CA14DB0420F022242A94322C03C022247B
:100D40002394312C89819A819E838D8397FF05C0DE
:100D50009195819591099E838D832D813E81319559
:100D6000219531093C832B83E614F70428F08FEF9B
:100D70009FEF9A83898304C021E030E03A8329837E
:100D800048018D819E81881A990AA201B701C60186
:100D900060DDC401880F991F2B813C818217930766
:100DA00064F0CA14DB0499F02D813E81821A930A03
:100DB000C20CD31C0817190744F3E614F70439F0E2
:100DC000800E911E89819A81E80EF91EDECF26964B
:100DD0000FB6F894DEBF0FBECDBFDF91CF911F914C
:100DE0000F91FF90EF90DF90CF90BF90AF909F90CA
:100DF0008F907F906F905F904F903F902F900895CD
:100E0000AF92BF92CF92DF92EF92FF920F931F9318
:100E1000CF93DF937C016B01EA01590198011CDF3C
:100E2000B501615071096C0D7D1D9801AE01C701BE
:100E300013DF9801A501B601C70130DFCE0101978C
:100E40009801A501B6018E0D9F1DDF91CF911F91D5
:100E50000F91FF90EF90DF90CF90BF90AF901ECF9B
:100E60002F923F924F925F926F927F928F929F92BA
:100E7000AF92BF92CF92DF92EF92FF920F931F93A8
:100E8000CF93DF931C012B01690150E0002711274C
:100E9000041B150BC1E0D0E0C41BD50BCC0FDD1F2C
:100EA000E12CF12CA6015701A40CB51CB5013101B0
:100EB000601A710AC301CDDCA601B5014801820C9C
:100EC000931CC401C6DCA6015201AE18BF08B501CF
:100ED000C401BFDCA601B501C301BBDCEC16FD06F5
:100EE000B4F08FEFE81AF80AC701880F991F01962E
:100EF0008C0F9D1F22273327201B310BE216F30690
:100F000039F40C171D074CF0C0E0D0E001C0CE0151
:100F10000C171D0714F0EC01C5CF0F5F1F4F980190
:100F2000220F331F2F5F3F4F820F931F10161106A2
:100F300094F7DF91CF911F910F91FF90EF90DF9089
:100F4000CF90BF90AF909F908F907F906F905F9069
:100F50004F903F902F9008954F925F926F927F92A3
:100F60008F929F92AF92BF92CF92DF92EF92FF92B9
:100F70000F931F93CF93DF93EC015B014A0139017B
:100F800028018601ADDE9701A201B301C401A8DEEC
:100F90009501AE01B701C201A3DEDF91CF911F9190
:100FA0000F91FF90EF90DF90CF90BF90AF909F9008
:100FB0008F907F906F905F904F900895CF93C82F40
:100FC0008A3011F48DE0FADF5D9BFECFCCB980E072
:100FD00090E0CF910895CF92DF92EF92FF920F931E
:100FE0001F93A8950FEF1FEF21E430E04FE550E08D
:100FF00065E070E085E090E003DFA89521E430E053
:101000004FE550E06BE470E085E090E0F9DE2BE422
:1010100030E04FE550E061E970E085E090E0F0DE1F
:10102000A3E2EA2EA5E0FA2E01E02FE130E04FEF37
:101030005FEF60E570E082E190E07BDDBEE1EB2EEA
:10104000B5E0FB2E2FE130E04FEF5FEF6AE570E097
:1010500083E290E06EDD0FEF1FEF21E430E04FE51B
:1010600050E065E070E08CED90E0CADE21E430E015
:101070004FE550E06BE470E08CED90E0C1DE2BE4D6
:1010800030E04FE550E061E970E08CED90E0B8DED3
:1010900013E2E12E15E0F12E01E02FE130E04FEFF9
:1010A0005FEF60E570E08BEE90E043DD88E1E82ED5
:1010B00085E0F82E2FE130E04FEF5FEF6AE570E05A
:1010C0008CEF90E036DD99E4E92E92E0F92E2FE1E5
:1010D00030E04FEF5FEF66EE70E08AE090E029DDF0
:1010E000A8958091120690911306019709F04FC0C0
:1010F0000FE110E024E430E048E550E064E970E0FE
:1011000088E090E021DC2CE430E04EE650E06CE832
:1011100070E089E690E018DC24E430E048E550E037
:1011200064E970E080EE90E00FDC20EE37E048E20A
:1011300064EB70E080EA90E093DE20EE37E047E277
:1011400064EB70E080EA90E08BDE20EE37E04BE26B
:1011500064EB70E080EA90E083DE20EE37E045E269
:1011600064EB70E080EA90E07BDEE0EECE2EE7E01C
:10117000DE2EF4EBEF2EF12C07EB10E028EC30E044
:1011800044E950E060EA70E084E990E0E5DEA8958B
:101190008091120690911306892B09F051C00FE13E
:1011A00010E024E430E048E550E064E970E088E0D5
:1011B00090E0CADB2CE430E04EE650E06CE870E0F2
:1011C00089E690E0C1DB24E430E048E550E064E9E2
:1011D00070E080EE90E0B8DB20E038EF48E264EBAE
:1011E00070E080EA90E03CDE20E038EF47E264EB1C
:1011F00070E080EA90E034DE20E038EF4BE264EB10
:1012000070E080EA90E02CDE20E038EF45E264EB0D
:1012100070E080EA90E024DE00E018EF23E230E0A6
:1012200045E050E065EA70E086E990E08DDB23E27E
:1012300030E045E050E065EA70E085EA90E084DB6C
:10124000A8958091140690911506892B79F4A8959C
:101250007EE0E72E75E0F72E01E02FE130E04FEF62
:101260005FEF63E270E08AE090E063DC8091140657
:10127000909115060197E1F4A89557ECE52E55E0FD
:10128000F52E01E02FE130E04FEF5FEF64E170E019
:1012900084E190E04EDC61ECE62E65E0F62E2FE175
:1012A00030E04FEF5FEF68E270E08EE190E041DC0C
:1012B000A89580911406909115060297E1F4A895DF
:1012C0003AEBE32E35E0F32E01E02FE130E04FEF73
:1012D0005FEF64E170E084E190E02BDC41ECE42E10
:1012E00045E0F42E2FE130E04FEF5FEF68E270E071
:1012F0008EE190E01EDCA895809114069091150671
:10130000039779F4A89523EBE22E25E0F22E01E075
:101310002FE130E04FEF5FEF63E270E089E190E0B2
:1013200008DCA8958091140690911506049779F42D
:10133000A89594EDE92E94E0F92E01E02FE130E03C
:101340004FEF5FEF63E270E08FE090E0F2DBA89593
:1013500080911406909115060597E1F4A8950EEC7E
:10136000E02E04E0F02E01E02FE130E04FEF5FEFE0
:1013700064E170E089E190E0DCDB84ECE82E84E05D
:10138000F82E2FE130E04FEF5FEF63E270E08FE087
:1013900090E0CFDBA89580911406909115060697F2
:1013A000E1F4A895BEECEB2EB4E0FB2E01E02FE1BA
:1013B00030E04FEF5FEF64E170E089E190E0B9DB8E
:1013C00012EBE12E14E0F12E2FE130E04FEF5FEF52
:1013D00063E270E08FE190E0ACDBA89580911406A9
:1013E00090911506079779F4A895A9E9EA2EA4E04B
:1013F000FA2E01E02FE130E04FEF5FEF63E270E0A3
:101400008FE090E096DB8091140690911506892B71
:1014100009F048C0A895E09173068E2F90E08830BF
:10142000910508F03FC0FC01EA5BFF4F0C942F3F91
:10143000F4E9EF2EF4E0FF2E04C0EFE8EE2EE4E036
:10144000FE2E02E02FE130E04FEF5FEF6EE170E043
:101450008BEE90E026C075E8E72E74E0F72E18C0FA
:101460006BE7E62E64E0F62E13C051E7E52E54E05C
:10147000F52E0EC047E6E42E44E0F42E09C03DE50B
:10148000E32E34E0F32E04C023E5E22E24E0F22E16
:1014900001E02FE130E04FEF5FEF6EE170E086EEAC
:1014A00090E047DB8091140690911506019701F5B5
:1014B000A89580911D06813069F038F08230C1F422
:1014C00001E7E02E04E0F02E09C095E8E92E94E053
:1014D000F92E04C08BE7E82E84E0F82E01E02FE11E
:1014E00030E04FEF5FEF6EE170E086EE90E021DBE1
:1014F0008091140690911506029701F5A8958091A8
:101500002406813069F038F08230C1F4A1E7EA2E78
:10151000A4E0FA2E09C015E8E12E14E0F12E04C073
:10152000BBE7EB2EB4E0FB2E01E02FE130E04FEF04
:101530005FEF6EE170E086EE90E0FBDA80911406DA
:1015400090911506039779F4A895FFEDEF2EF4E03E
:10155000FF2E01E02FE130E04FEF5FEF6EE170E032
:101560008EEE90E0E6DA80911406909115060497CD
:1015700001F5A89580917E06813069F038F08230BF
:10158000C1F461E7E62E64E0F62E09C0E5E8EE2E30
:10159000E4E0FE2E04C07BE7E72E74E0F72E01E0C6
:1015A0002FE130E04FEF5FEF6EE170E086EE90E00C
:1015B000C0DA8091140690911506059701F5A8955B
:1015C00080917206813069F038F08230C1F431E7E1
:1015D000E32E34E0F32E09C055E8E52E54E0F52E55
:1015E00004C04BE7E42E44E0F42E01E02FE130E0AC
:1015F0004FEF5FEF6EE170E086EE90E09ADA809157
:10160000140690911506069701F5A89580916F062E
:10161000813069F038F08230C1F481E7E82E84E04F
:10162000F82E09C025E8E22E24E0F22E04C09BE744
:10163000E92E94E0F92E01E02FE130E04FEF5FEF6B
:101640006EE170E086EE90E074DA8091140690917D
:101650001506079709F4A8951F910F91FF90EF9039
:10166000DF90CF900895CF92DF92EF92FF920F9389
:101670001F93A89500EE17E021E430E048EC50E01D
:101680006AEA70E085E090E05FD90FEF1FEF21E498
:1016900030E048EC50E063E270E085E090E0B0DBE1
:1016A00087E6E82E82E0F82E01E02FE130E040EE00
:1016B00057E06CE370E088E290E03BDA0FEF1FEF59
:1016C00020E530E040E550E065E070E08BEE90E032
:1016D00097DB90EEC92E97E0D92E24E1E22EF12C73
:1016E00003E111E026E430E041E351E066E470E01C
:1016F00085EF90E031DC37E1E32EF12C24E430E09B
:101700004FE251E064E470E087EF90E025DC0FEFFA
:101710001FEF20E530E040E550E064E670E08BEE3E
:1017200090E06EDB45EAE42EF12C03E111E023E7C3
:1017300030E041E351E063E770E085EF90E00CDCDE
:1017400053EAE52EF12C25E730E04FE251E065E762
:1017500070E087EF90E000DC66E3E62E65E0F62EB1
:1017600002E020EE37E040E050E068EC70E08DE20F
:1017700090E0DFD91F910F91FF90EF90DF90CF9015
:101780000895CF92DF92EF92FF920F931F93A89547
:1017900000EE17E021E430E048EC50E06AEA70E047
:1017A00085E090E0D1D80FEF1FEF21E430E048EC66
:1017B00050E063E270E085E090E022DB83EAE82E0F
:1017C00084E0F82E01E02FE130E040EE57E06CE3DA
:1017D00070E088E290E0ADD90FEF1FEF20E530E038
:1017E00040E550E065E070E08BEE90E009DB90EEC4
:1017F000C92E97E0D92E24E1E22EF12C03E111E06D
:1018000026E430E041E351E066E470E085EF90E0EB
:10181000A3DB37E1E32EF12C24E430E04FE251E08A
:1018200064E470E087EF90E097DB0FEF1FEF20E5B7
:1018300030E040E550E064E670E08BEE90E0E0DA06
:1018400045EAE42EF12C03E111E023E730E041E327
:1018500051E063E770E085EF90E07EDB53EAE52E30
:10186000F12C25E730E04FE251E065E770E087EFCB
:1018700090E072DB6FECE62E65E0F62E02E020EEE3
:1018800037E040E050E068EC70E08DE290E051D944
:101890001F910F91FF90EF90DF90CF900895CF921E
:1018A000DF92EF92FF920F931F93A89500EE17E03F
:1018B00021E430E048EC50E06AEA70E085E090E036
:1018C00043D80FEF1FEF21E430E048EC50E063E233
:1018D00070E085E090E094DA82E4E82E84E0F82E6F
:1018E00001E02FE130E040EE57E06CE370E088E289
:1018F00090E01FD90FEF1FEF20E530E040E550E00A
:1019000065E070E08BEE90E07BDA90EEC92E97E018
:10191000D92E24E1E22EF12C03E111E026E430E09F
:1019200041E351E066E470E085EF90E015DB37E1DC
:10193000E32EF12C24E430E04FE251E064E470E067
:1019400087EF90E009DB0FEF1FEF20E530E040E587
:1019500050E064E670E08BEE90E052DA45EAE42E67
:10196000F12C03E111E023E730E041E351E063E7CC
:1019700070E085EF90E0F0DA53EAE52EF12C25E7F0
:1019800030E04FE251E065E770E087EF90E0E4DAA5
:1019900067E4E62E65E0F62E02E020EE37E040E058
:1019A00050E068EC70E08DE290E0C3D81F910F9199
:1019B000FF90EF90DF90CF900895CF93DF9300D00A
:1019C00000D0CDB7DEB7809163001C821B821A82E3
:1019D0001982BE016F5F7F4FCE0103960E94923D38
:1019E0008B819C818431954068F489819A81843A05
:1019F000964040F489819A818D32914018F082E0BE
:101A000080933C068B819C818937954090F08B8137
:101A10009C81843C994068F489819A81843A9640FB
:101A200040F489819A818D32914018F083E080934F
:101A30003C068B819C8189329A4068F089819A8129
:101A400084379E4040F489819A81813D974018F007
:101A500081E080933C068B819C81863F994060F4B5
:101A60008B819C818134964038F089819A81813DB7
:101A7000974010F010923C0680913C060F900F901A
:101A80000F900F90DF91CF910895CF92DF92EF9258
:101A9000FF920F931F93A89500EE17E021E430E02A
:101AA00048EC50E06AEA70E085E090E00E94A4040F
:101AB0000FEF1FEF21E430E048EC50E063E270E00C
:101AC00085E090E09DD920E530E040E550E065E01C
:101AD00070E08BEE90E094D9F0EECF2EF7E0DF2EA1
:101AE000A4E1EA2EF12C03E111E026E430E041E329
:101AF00051E066E470E085EF90E02EDAB7E1EB2E7E
:101B0000F12C24E430E04FE251E064E470E087EF30
:101B100090E022DA0FEF1FEF20E530E040E550E0E3
:101B200064E670E08BEE90E06BD915EAE12EF12CC3
:101B300003E111E023E730E041E351E063E770E0C7
:101B400085EF90E009DA83EAE82EF12C25E730E012
:101B50004FE251E065E770E087EF90E0FDD99FEC40
:101B6000E92E95E0F92E02E020EE37E040E050E06B
:101B700068EC70E08CE390E00E9499058091140677
:101B800090911506892B09F048C0E09173068E2FBD
:101B900090E08830910508F040C0FC01E25BFF4F07
:101BA0000C942F3FE4E9EE2EE4E0FE2E04C07FE823
:101BB000E72E74E0F72E02E02FE130E04FEF5FEF09
:101BC00065E070E086E490E026C065E8E62E64E01B
:101BD000F62E18C05BE7E52E54E0F52E13C041E762
:101BE000E42E44E0F42E0EC037E6E32E34E0F32E6C
:101BF00009C02DE5E22E24E0F22E04C093E5E92E83
:101C000094E0F92E02E02FE130E04FEF5FEF65E066
:101C100070E08EE190E00E94990580911406909109
:101C20001506019701F580911D06813069F038F0A5
:101C30008230C9F411E7E12E14E0F12E09C085E8E5
:101C4000E82E84E0F82E04C00BE7E02E04E0F02E2E
:101C500002E02FE130E04FEF5FEF65E070E08EE1F2
:101C600090E00E94990580911406909115060297C4
:101C700001F580912406813069F038F08230C9F492
:101C8000F1E7EF2EF4E0FF2E09C0B5E8EB2EB4E04B
:101C9000FB2E04C0ABE7EA2EA4E0FA2E02E02FE10F
:101CA00030E04FEF5FEF65E070E08EE190E00E9482
:101CB00099058091140690911506049701F580917D
:101CC0007E06813069F038F08230C9F461E7E62E93
:101CD00064E0F62E09C0E5E8EE2EE4E0FE2E04C036
:101CE0007BE7E72E74E0F72E02E02FE130E04FEFC4
:101CF0005FEF65E070E08EE190E00E9499058091D1
:101D0000140690911506059701F5809172068130B1
:101D100069F038F08230C9F431E7E32E34E0F32E75
:101D200009C055E8E52E54E0F52E04C04BE7E42E3B
:101D300044E0F42E02E02FE130E04FEF5FEF65E08A
:101D400070E08EE190E00E949905809114069091D8
:101D50001506069701F580916F06813069F038F01D
:101D60008230C9F481E7E82E84E0F82E09C025E826
:101D7000E22E24E0F22E04C09BE7E92E94E0F92E37
:101D800002E02FE130E04FEF5FEF65E070E08EE1C1
:101D900090E00E9499051F910F91FF90EF90DF90C6
:101DA000CF900895EF92FF920F931F9380910B06AF
:101DB00090910C060A97A8F48091E20581110CC05D
:101DC0000FE110E02CE330E044E650E06BE470E01B
:101DD0008EE690E00E94A40481E08093E2051092D8
:101DE000160680910B0690910C060A978A3591058C
:101DF000A8F48091160681110CC00FE110E02CE3CD
:101E000030E044E650E06BE470E08EE690E00E9443
:101E1000A40481E0809316061092E20580910B06DF
:101E200090910C0684369105A0F0809116068130C1
:101E300061F40FE110E02CE330E044E650E06BE4A5
:101E400070E08EE690E00E94A404109216061092B4
:101E5000E2058091120690911306019779F4E090C3
:101E60000B06F0900C0603E02FE130E04FEF5FEF40
:101E700064E670E082E890E00E94DF05809112063F
:101E800090911306892B79F4E0900B06F0900C06E4
:101E900003E02FE130E040E058EF64E670E082E8D4
:101EA00090E00E94DF051F910F91FF90EF90089541
:101EB000EF92FF920F931F938091400690914106FD
:101EC0000A97A8F480910A06811111C00FE110E071
:101ED00027E330E048E550E06BE970E088E090E00F
:101EE0000E94A40481E080930A06109270068091FB
:101EF00040069091410684369105D8F480910B06F6
:101F000090910C060A97A8F080917006811111C07B
:101F10000FE110E027E330E048E550E06BE970E0C6
:101F200088E090E00E94A40481E080937006109203
:101F30000A06809140069091410684369105A0F0F2
:101F400080917006813061F40FE110E027E330E00A
:101F500048E550E06BE970E088E090E00E94A4045E
:101F60001092700610920A06E0904006F09041062A
:101F700003E02FE130E04FEF5FEF64EB70E08FE0C4
:101F800090E00E94DF051F910F91FF90EF90089560
:101F9000EF92FF920F931F9380912D0690912E0642
:101FA0000A97A8F48091110681110CC00FE110E08E
:101FB00024E230E04AE550E064E670E088E090E03A
:101FC0000E94A40481E0809311061092280680915B
:101FD0002D0690912E060A978A359105A8F48091D6
:101FE000280681110CC00FE110E024E230E04AE540
:101FF00050E064E670E088E090E00E94A40481E094
:10200000809328061092110680912D0690912E063D
:1020100084369105A1F480912806813061F40FE1A6
:1020200010E024E230E04AE550E064E670E088E049
:1020300090E00E94A4041092110610922806E090ED
:102040002D06F0902E0603E02FE130E04FEF5FEF1A
:102050006EE670E084E190E00E94DF0580917F06EB
:10206000909180060A97A8F480917906811111C099
:102070000FE110E024E230E04AE550E064E670E071
:102080008FED90E00E94A40481E080937906109285
:10209000420680917F06909180060A978A359105C5
:1020A000A8F480914206811111C00FE110E024E2F2
:1020B00030E04AE550E064E670E08FED90E00E9489
:1020C000A40481E08093420610927906E0907F0696
:1020D000F090800684E6E816F10421F41092790667
:1020E0001092420603E02FE130E04FEF5FEF6EE623
:1020F00070E089EE90E00E94DF051F910F91FF9044
:10210000EF900895CF93DF9300D000D0CDB7DEB726
:10211000809163001C821B821A821982BE016F5F4C
:102120007F4FCE0103960E94923D8B819C81853C1E
:102130009940A0F0A89589819A81843C994070F4D7
:10214000A89589819A818D3D954040F0A89581E0C0
:1021500090E09093130680931206A8950F900F902D
:102160000F900F90DF91CF910895CF93DF9300D020
:1021700000D0CDB7DEB7A895809163001C821B828A
:102180001A821982BE016F5F7F4FCE0103960E94B3
:10219000923D8B819C81853C9940A8F089819A81F0
:1021A000843C994080F489819A818D3D954058F016
:1021B00010921306109212068FE19EE40197F1F738
:1021C00000C00000A8950F900F900F900F90DF9126
:1021D000CF9108957F928F929F92AF92BF92CF92AC
:1021E000DF92EF92FF920F931F93CF93DF93EC0157
:1021F0006B015A014901702EA8958091E5059091D7
:10220000E6050A97A8F480917406811111C00FE1C8
:1022100010E02EE130E044E650E065507109CE0157
:1022200044970E94A40481E08093740610923506BE
:102230008091E5059091E6050A978A359105C0F4ED
:1022400080913506811114C00FE110E02EE130E0DD
:1022500044E650E0B60165507109CE0144970E94F2
:10226000A40481E0809335061092740610920D0646
:102270008091E5059091E60584369105C0F0809146
:102280000D06811114C00FE110E02EE130E044E6AC
:1022900050E0B60165507109CE0144970E94A40434
:1022A00081E080930D061092350610927406E0903E
:1022B000E505F090E605072D9401A501B601CE01D4
:1022C0000E94DF05A895DF91CF911F910F91FF909C
:1022D000EF90DF90CF90BF90AF909F908F907F90C6
:1022E0000895A89583EB92E00E944A42813069F4F8
:1022F000A49AAC9AA8952FEF82E597E021508040F0
:102300009040E1F700C00000AC98A8950895A8950A
:1023100080913206813019F5A49AAC9A2FEF82E5AC
:1023200097E0215080409040E1F700C00000A89560
:10233000AC982FEF82E597E0215080409040E1F784
:1023400000C00000A895AC9A2FEF82E597E02150DD
:1023500080409040E1F700C00000A895AC98089537
:10236000A89580913206813009F047C0A49AAC9AB2
:10237000A8952FEF82E597E0215080409040E1F74B
:1023800000C00000A895AC98A8952FEF82E597E0D3
:10239000215080409040E1F700C00000A895AC9A21
:1023A000A8952FEF82E597E0215080409040E1F71B
:1023B00000C00000A895AC98A8952FEF82E597E0A3
:1023C000215080409040E1F700C00000A895AC9AF1
:1023D0002FEF82E597E0215080409040E1F700C068
:1023E0000000A895AC982FEF82E597E0215080403F
:1023F0009040E1F700C00000A8950895A8951092BC
:102400002F06109221061092E005109245061092B8
:102410001E06109210061092310610922706109296
:102420003F061092E10583EB92E00E944A428093BE
:102430003206A89584EB92E00E94524290932306C4
:1024400080932206A8958091140690911506892BF9
:1024500051F5A895E09173068E2F90E08830910594
:1024600010F5FC01EA5AFF4F4EE150E00C942F3F6B
:1024700064E972E014C066E772E011C068E572E0DA
:102480000EC06AE372E00BC06CE172E008C06EEF50
:1024900071E005C060EE71E002C062EC71E08BEEAD
:1024A00095E00E943A42A8958091140690911506F5
:1024B0000197D1F4A89580911D06813069F038F01C
:1024C000823091F44EE150E068E671E009C04EE1DF
:1024D00050E064EA71E004C04EE150E066E871E06B
:1024E0008BEE95E00E943A42A89580911406909157
:1024F00015060297D1F4A89580912406813069F0E1
:1025000038F0823091F44EE150E06EE071E009C0A5
:102510004EE150E06AE471E004C04EE150E06CE24C
:1025200071E08BEE95E00E943A42A89580911406E6
:10253000909115060497C9F480917E06813069F068
:1025400038F0823091F44EE150E064EB70E009C065
:102550004EE150E060EF70E004C04EE150E062ED0B
:1025600070E08BEE95E00E943A42A89580911406A7
:10257000909115060597C9F480917206813069F033
:1025800038F0823091F44EE150E06AE570E009C025
:102590004EE150E066E970E004C04EE150E068E7CB
:1025A00070E08BEE95E00E943A42A8958091140667
:1025B000909115060697C9F480916F06813069F0F5
:1025C00038F0823091F44EE150E060E070E009C0F4
:1025D0004EE150E06CE370E004C04EE150E06EE18B
:1025E00070E08BEE95E00E943A42A89587EC90E06F
:1025F0000197F1F700C000008091EB059091EC0588
:102600009093DF058093DE058091ED059091EE05B6
:1026100090933406809333068091EF059091F005F6
:1026200090937C0680937B068091F1059091F20552
:1026300090931C0680931B068091F30580934806B7
:102640008091F5059091F60590931A0680931906EE
:102650008091F7059091F80590932C0680932B06B6
:102660008091F9059091FA0590932A0680932906A6
:102670008091FB058093DA058091FD059091FE0520
:1026800090936C0680936B068091FF0590910006F5
:102690009093470680934606809114069091150604
:1026A000079741F4809101069091020690931506D8
:1026B00080931406809103069091040690936A0615
:1026C0008093690680910506909106069093EA052D
:1026D0008093E905809107069091080690930F0674
:1026E00080930E06A89508951092800610927F069A
:1026F000BC9A80917F06880F81BF10922E0610929F
:102700002D06139A80912D06880F8093860028DE6F
:102710008DE490E0909376068093750681E090E0DA
:1027200090931306809312060895CF93BC9A8091DC
:102730007F06880F81BF139A80912D06880F8093A2
:1027400086008091140690911506892B09F0F3C13B
:102750004091E5055091E60520911B0630911C063D
:10276000429FC001439F900D529F900D11246AE03B
:1027700070E00E941B3F7093440660934306809173
:102780002D0690912E068536910530F084E690E076
:1027900090932E0680932D062091290630912A06CB
:1027A00080912D0690912E062817390720F430933A
:1027B0002E0620932D0680912F06811113C0809143
:1027C0004006909141068233910538F484E690E00A
:1027D00090932E0680932D0605C0C29719F081E0D4
:1027E00080932F0680912F06E0913306F0913406F6
:1027F000813051F56E177F0738F5409140065091B2
:10280000410680912D0690912E0646175707B8F481
:1028100001962817390728F090932E0680932D06ED
:1028200004C030932E0620932D0680912D069091A2
:102830002E068536910540F084E690E001C00197B0
:1028400090932E0680932D06E617F70798F5409192
:102850004006509141064E175F07C8F480912D063F
:1028600090912E0601968536910510F084E690E051
:1028700090932E0680932D0680912D0690912E0622
:102880002817390720F430932E0620932D06E417DD
:10289000F50780F480912D0690912E064E1B5F0B5C
:1028A0004B30510510F4019701C00B9790932E0601
:1028B00080932D06C0914806C130D1F48091210645
:1028C000811116C020910B0630910C0680911906DB
:1028D00090911A062817390759F480914006909173
:1028E00041069093340680933306FBDCC0932106A7
:1028F000C091DA05C13009F58091E00581111DC054
:1029000080910B0690910C0620916B0630916C061D
:10291000821B930B059788F420913306309134067F
:102920008091460690914706820F931F909334063C
:1029300080933306D6DCC093E00580914506811173
:102940001CC080910B0690910C06209119063091C5
:102950001A06821B930B029780F482E390E0909317
:10296000800680937F0681E0809345068093100661
:1029700080914806811101C0B4DC20911906309184
:102980001A06609177067091780640917B06509107
:102990007C06649FC001659F900D749F900D11246B
:1029A0006AE070E00E941B3F620F731F7093DD05A9
:1029B0006093DC05E0917F06F09180064091DE0592
:1029C0005091DF054617570720F45093DD054093DB
:1029D000DC0580912B0690912C068E179F0720F422
:1029E0009093800680937F0680910B0690910C0651
:1029F0002817390700F520913F0621111CC08417C4
:102A00009507C8F46091DC057091DD0520917F0683
:102A1000309180068617970740F42F5F3F4F253689
:102A2000310528F024E630E002C02150310930930E
:102A3000800620937F064817590768F520917F0686
:102A400030918006841B950B069718F421503109AC
:102A500002C02B5031093093800620937F0680916D
:102A6000E105811106C053DC81E080932706809345
:102A7000E1052091E7053091E805809122069091CB
:102A800023068217930738F42FDE81E090E09093BD
:102A900013068093120680911E0681114CC040914E
:102AA000690650916A068091190690911A0684175A
:102AB000950708F040C0E0910B06F0910C064E1708
:102AC0005F0729F481E080933F068093310680916F
:102AD0003F06813081F56091E3057091E405209116
:102AE000E9053091EA056217730798F480917F0633
:102AF00090918006E417F50738F401968536910524
:102B000020F084E690E001C00197909380068093C6
:102B10007F062617370778F410923F0680917706D4
:102B200090917806821B930B90937806809377069A
:102B300081E080931E0680911406909115060197FE
:102B400009F001C110922E0610922D0680914506C3
:102B500081111BC020910B0630910C068091190643
:102B600090911A068217930780F482E390E0909385
:102B7000800680937F0681E080934506809310064F
:102B800080914806811101C0ACDB2091190630917B
:102B90001A06609177067091780640917B065091F5
:102BA0007C06649FC001659F900D749F900D112459
:102BB0006AE070E00E941B3F620F731F7093DD0597
:102BC0006093DC05E0917F06F09180064091DE0580
:102BD0005091DF054617570720F45093DD054093C9
:102BE000DC0580912B0690912C068E179F0720F410
:102BF0009093800680937F0680910B0690910C063F
:102C00002817390700F520913F0621111CC08417B1
:102C10009507C8F46091DC057091DD0520917F0671
:102C2000309180068617970740F42F5F3F4F253677
:102C3000310528F024E630E002C0215031093093FC
:102C4000800620937F064817590768F520917F0674
:102C500030918006841B950B069718F4215031099A
:102C600002C02B5031093093800620937F0680915B
:102C7000E105811106C04BDB81E08093270680933C
:102C8000E1052091E7053091E805809122069091B9
:102C900023068217930738F427DD81E090E09093B4
:102CA00013068093120680911E0681114CC040913C
:102CB000690650916A068091190690911A06841748
:102CC000950708F040C0E0910B06F0910C064E17F6
:102CD0005F0729F481E080933F068093310680915D
:102CE0003F06813081F56091E3057091E405209104
:102CF000E9053091EA056217730798F480917F0621
:102D000090918006E417F50738F401968536910511
:102D100020F084E690E001C00197909380068093B4
:102D20007F062617370778F410923F0680917706C2
:102D300090917806821B930B909378068093770688
:102D400081E080931E0680911406909115060297EB
:102D500009F00FC11092800610927F06C0914806BC
:102D6000C130D1F480912106811116C020910B064B
:102D700030910C068091190690911A062817390790
:102D800059F48091400690914106909334068093C7
:102D90003306A7DAC09321064091E5055091E60578
:102DA00020911B0630911C06429FC001439F900D4D
:102DB000529F900D11246AE070E00E941B3F7093B7
:102DC00044066093430680912D0690912E06853629
:102DD000910530F084E690E090932E0680932D06C6
:102DE0008091290690912A0620912D0630912E0679
:102DF0008217930720F490932E0680932D0620913E
:102E00002F06211114C02091400630914106263929
:102E1000310538F424E630E030932E0620932D0659
:102E200006C02639310519F021E020932F062091A4
:102E30002F064091330650913406213061F5641716
:102E4000750748F5E0914006F091410620912D0666
:102E500030912E06E617F707C0F42F5F3F4F821719
:102E6000930728F030932E0620932D0604C09093EC
:102E70002E0680932D0620912D0630912E062536A4
:102E8000310548F024E630E002C02150310930938A
:102E90002E0620932D064617570708F06AC020918A
:102EA000480621112CC0209140063091410624177C
:102EB0003507D0F460912D0670912E066F5F7F4F1D
:102EC0006536710510F064E670E070932E0660932D
:102ED0002D0660912D0670912E068617970720F417
:102EE00090932E0680932D064217530708F041C099
:102EF00080912D0690912E06241B350B30C0213079
:102F0000C1F520910B0630910C0660911906709165
:102F10001A0626173707D0F440912D0650912E0639
:102F20004F5F5F4F4536510510F044E650E0509337
:102F30002E0640932D0640912D0650912E068417A3
:102F4000950720F490932E0680932D066217730741
:102F500080F480912D0690912E06261B370B2B3086
:102F6000310510F4019701C00B9790932E068093C2
:102F70002D0680911406909115068430910521F05C
:102F80008530910509F0DAC04091E5055091E605DC
:102F900020911B0630911C06429FC001439F900D5B
:102FA000529F900D11246AE070E00E941B3F7093C5
:102FB00044066093430680912D0690912E06853637
:102FC000910530F084E690E090932E0680932D06D4
:102FD000E0912906F0912A0680912D0690912E0607
:102FE000E817F90720F4F0932E06E0932D062091C0
:102FF0002F068091400690914106211110C086391C
:10300000910538F424E630E030932E0620932D0607
:1030100006C08639910519F021E020932F062091F2
:103020002F064091330650913406213041F5641744
:10303000750728F520912D0630912E0686179707E3
:10304000C0F42F5F3F4FE217F30728F030932E06AE
:1030500020932D0604C0F0932E06E0932D062091B8
:103060002D0630912E062536310548F024E630E055
:1030700002C02150310930932E0620932D064617A9
:10308000570738F120912B0630912C0660917F066E
:10309000709180062617370720F43093800620931E
:1030A0007F064817590708F0FFC080917F0690916E
:1030B000800601969093800680937F068536910561
:1030C00008F4F2C084E690E09093800680937F0637
:1030D000EBC084179507D0F420912D0630912E0671
:1030E0002F5F3F4F2536310510F024E630E0309356
:1030F0002E0620932D0620912D0630912E06E217E4
:10310000F30720F4F0932E06E0932D064817590795
:1031100008F0B8CF20912D0630912E06BC01641B1B
:10312000750B6B30710538F02B50310930932E063A
:1031300020932D06A7CF21503109F8CF069709F02B
:10314000B3C04091E5055091E60520911B063091F2
:103150001C06429FC001439F900D529F900D112469
:103160006AE070E00E941B3F709344066093430640
:1031700080912D0690912E068536910530F084E6DB
:1031800090E090932E0680932D0620912906309191
:103190002A0680912D0690912E062817390720F4D3
:1031A00030932E0620932D0680912F06811114C096
:1031B00080914006909141068639910538F484E665
:1031C00090E090932E0680932D0606C086399105D7
:1031D00019F081E080932F0680912F06E09133064D
:1031E000F0913406813051F56E177F0738F5409124
:1031F00040065091410680912D0690912E0646176B
:103200005707B8F401962817390728F090932E062F
:1032100080932D0604C030932E0620932D068091B6
:103220002D0690912E068536910540F084E690E0BB
:1032300001C0019790932E0680932D06E617F7079D
:1032400098F540914006509141064E175F07C8F42B
:1032500080912D0690912E0601968536910510F0ED
:1032600084E690E090932E0680932D0680912D06A3
:1032700090912E062817390720F430932E062093BC
:103280002D06E417F50780F480912D0690912E0607
:103290004E1B5F0B4B30510510F4019701C00B978B
:1032A00090932E0680932D06CF91089563EC70E0E5
:1032B00084E992E00E946D4262EC71E086E992E05E
:1032C0000E946D4266E170E088E992E00E946D42E2
:1032D00066E170E08AE992E00E946D4261E070E090
:1032E0008CE992E00E946D42A8956EE670E08EE94E
:1032F00092E00E946D4264E670E080EA92E00E94F3
:103300006D4264E670E082EA92E00E946D4260E005
:1033100070E084EA92E00E946D42A89560E070E05F
:1033200086EA92E00E946D4260E070E088EA92E0F6
:103330000E946D4260E070E08AEA92E00E946D4275
:1033400060E070E08CEA92E00E946D4260E070E024
:103350008EEA92E00E946D4260E070E080EB92E0C5
:103360000E946D42A89566EE70E086E792E00E94AA
:103370006D4262EC71E088E792E00E946D4266E186
:1033800070E08AE792E00E946D4266E170E08CE7AF
:1033900092E00E946D4261E070E08EE792E00E9450
:1033A0006D42A89563E770E080E892E00E946D426C
:1033B00064E670E082E892E00E946D4264E670E0AC
:1033C00084E892E00E946D4260E070E086E892E05E
:1033D0000E946D4260E070E088E892E00E946D42D9
:1033E00060E070E08AE892E00E946D42A89560E09B
:1033F00070E08CE892E00E946D4260E070E08EE840
:1034000092E00E946D4260E070E080E992E00E94EC
:103410006D4260E070E082E992E00E946D42A89502
:1034200066EE70E088E592E00E946D4262EC71E029
:103430008AE592E00E946D4266E170E08CE592E0E0
:103440000E946D4266E170E08EE592E00E946D425E
:1034500061E070E080E692E00E946D42A89563E72B
:1034600070E082E692E00E946D4264E670E084E6DD
:1034700092E00E946D4264E670E086E692E00E946F
:103480006D4260E070E088E692E00E946D4260E08C
:1034900070E08AE692E00E946D4260E070E08CE6A7
:1034A00092E00E946D42A89560E070E08EE692E0A6
:1034B0000E946D4260E070E080E792E00E946D4201
:1034C00060E070E082E792E00E946D4260E070E0B0
:1034D00084E792E00E946D42A89566E970E08AE375
:1034E00092E00E946D4268EC70E08CE392E00E94F2
:1034F0006D4266E170E08EE392E00E946D4266E10B
:1035000070E080E492E00E946D4261E070E082E44D
:1035100092E00E946D42A89563E770E084E492E037
:103520000E946D4264E670E086E492E00E946D4283
:1035300064E670E088E492E00E946D4260E070E032
:103540008AE492E00E946D4260E070E08CE492E0D8
:103550000E946D4260E070E08EE492E00E946D4255
:10356000A89560E070E080E592E00E946D4260E026
:1035700070E082E592E00E946D4260E070E084E5D8
:1035800092E00E946D4260E070E086E592E00E9469
:103590006D42A8956EEB70E08CE192E00E946D4266
:1035A00068EC70E08EE192E00E946D4266E170E0AE
:1035B00080E292E00E946D4266E170E082E292E079
:1035C0000E946D4261E070E084E292E00E946D42F0
:1035D000A89564E670E086E292E00E946D4264E69F
:1035E00070E088E292E00E946D4264E670E08AE258
:1035F00092E00E946D4260E070E08CE292E00E94F6
:103600006D4260E070E08EE292E00E946D4260E008
:1036100070E080E392E00E946D42A89560E070E067
:1036200082E392E00E946D4260E070E084E392E009
:103630000E946D4260E070E086E392E00E946D427D
:1036400060E070E088E392E00E946D42A89566EE2B
:1036500070E08EEF91E00E946D4262EC71E080E0DC
:1036600092E00E946D4266E170E082E092E00E948A
:103670006D4266E170E084E092E00E946D4261E09C
:1036800070E086E092E00E946D42A89563E770E0EA
:1036900088E092E00E946D4264E670E08AE092E089
:1036A0000E946D4264E670E08CE092E00E946D4200
:1036B00060E070E08EE092E00E946D4260E070E0B9
:1036C00080E192E00E946D4260E070E082E192E071
:1036D0000E946D42A89560E070E084E192E00E9453
:1036E0006D4260E070E086E192E00E946D4260E031
:1036F00070E088E192E00E946D4260E070E08AE153
:1037000092E00E946D42A89566EE70E080EE91E036
:103710000E946D4262EC71E082EE91E00E946D4287
:1037200066E170E084EE91E00E946D4266E170E037
:1037300086EE91E00E946D4261E070E088EE91E0DB
:103740000E946D42A89563E770E08AEE91E00E94C6
:103750006D4264E670E08CEE91E00E946D4264E69A
:1037600070E08EEE91E00E946D4260E070E080EFCC
:1037700091E00E946D4260E070E082EF91E00E9473
:103780006D4260E070E084EF91E00E946D42A89588
:1037900060E070E086EF91E00E946D4260E070E0D2
:1037A00088EF91E00E946D4260E070E08AEF91E066
:1037B0000E946D4260E070E08CEF91E00E946D42EB
:1037C000A89563EC70E084EA91E00E946D4266E1A6
:1037D00070E088EA91E00E946D4261E070E08CEA5E
:1037E00091E00E946D426FE070E08EEA91E00E94ED
:1037F0006D42A89564E670E080EB91E00E946D4216
:1038000061E070E08AEB91E00E946D4263EC70E051
:103810008CEB91E00E946D426AE070E08EEB91E0EB
:103820000E946D42A89562EC71E08CE491E00E94E8
:103830006D4266E170E080E591E00E946D4261E0DA
:1038400070E082E591E00E946D426EE670E084E5F2
:1038500091E00E946D42A89564E670E088E591E0F1
:103860000E946D4262E070E080E691E00E946D424D
:1038700062EC71E082EF90E00E946D4266E170E0E0
:1038800084EF90E00E946D4262E170E086EF90E08C
:103890000E946D42A89564E670E08CEF90E00E9473
:1038A0006D4264E670E08EEF90E00E946D4264E04D
:1038B00070E086E091E00E946D426CE271E08CE085
:1038C00091E00E946D42A89562EC71E088E990E079
:1038D0000E946D4266E170E08AE990E00E946D42CC
:1038E00066E170E08CE990E00E946D4261E070E07A
:1038F0008EE990E00E946D42A8956EE670E080EA45
:1039000090E00E946D4264E670E082EA90E00E94DE
:103910006D4264E670E084EA90E00E946D4265E0EA
:1039200070E08CEA90E00E946D42A89562EC71E034
:103930008EE390E00E946D4266E170E082E490E0E8
:103940000E946D4261E070E084E490E00E946D426C
:103950006EE670E086E490E00E946D42A89564E611
:1039600070E08AE490E00E946D4266E070E082E5DB
:1039700090E00E946D4263EC70E084E992E00E9466
:103980006D42A89508956FE070E088EB92E00E9488
:103990006D426FE070E086EB92E00E946D426FE056
:1039A00070E084EB92E00E946D4261E083EB92E074
:1039B0000E94604261E082EB92E00C9460428FB919
:1039C000779BFECF8FB10895CF93A39AAB9AAB9814
:1039D00080E0F5DFC82F80E0F2DFAB9A6C2F70E05B
:1039E000762F6627682B687F7F7723E0769567952B
:1039F0002A95E1F780E090E00E942A3E20E030E046
:103A000040E85EE30E94903E0E94FE3D70930C06EB
:103A100060930B06CB01CF910895CF93A79AAF9AED
:103A2000AF9880E0CCDFC82F80E0C9DFAF9A6C2F61
:103A300070E0762F6627682B687F7F7723E0769586
:103A400067952A95E1F780E090E00E942A3E20E009
:103A500030E040E85EE30E94903E0E94FE3D70939D
:103A6000410660934006CB01CF91089580E091E03C
:103A7000909385068093840680910C068F938091A5
:103A80000B068F938EE091E09F938F930E946A3F85
:103A90008DE08A95F1F700008091E6058F93809183
:103AA000E5058F9388E191E09F938F930E946A3F91
:103AB0009DE09A95F1F7000080912E068F938091FA
:103AC0002D068F9382E291E09F938F930E946A3F2D
:103AD0008DE08A95F1F70000809180068F938091A8
:103AE0007F068F938DE291E09F938F930E946A3FB0
:103AF0009DE09A95F1F7000087E391E09F938F9303
:103B00000E946A3F8DE08A95F1F70000809141069E
:103B10008F93809140068F938FE391E09F938F93D3
:103B20000E946A3FA8958DB79EB746960FB6F89447
:103B30009EBF0FBE8DBF8091120690911306892BF8
:103B400041F488E491E09F938F930E946A3F0F9025
:103B50000F90A8958091120690911306019741F459
:103B60008FE491E09F938F930E946A3F0F900F9094
:103B70009DE09A95F1F70000E0911406F09115068A
:103B8000E830F10508F09CC0E25AFF4F0C942F3F3B
:103B900086E591E09F938F930E946A3FA8950F90CE
:103BA0000F90E09173068E2F90E08830910508F019
:103BB00087C0FC01EA59FF4F0C942F3F85E691E046
:103BC00071C085E791E06EC08DEA91E06BC08CEB2F
:103BD00091E068C08BEC91E065C08AED91E09F9325
:103BE0008F930E946A3FA8950F900F9080911D06B9
:103BF000813009F452C008F44DC0823009F450C03D
:103C000008958AEE91E09F938F930E946A3FA89552
:103C10000F900F9080912406813009F43EC0D0F1BE
:103C2000823009F43DC008958BEF91E042C089E0F5
:103C300092E09F938F930E946A3FA8950F900F90F8
:103C400080917E06813049F128F1823049F1089552
:103C50008AE192E09F938F930E946A3FA8950F900C
:103C60000F90809172068130C1F0A0F08230C1F0D7
:103C700008958DE292E09F938F930E946A3FA895EA
:103C80000F900F9080916F06813039F018F08230DC
:103C900039F0089580E891E005C08FE891E002C016
:103CA0008EE991E09F938F930E946A3F07C08FE354
:103CB00092E09F938F930E946A3FA8950F900F9078
:103CC0000895CF92DF92EF92FF920F931F93CF93BD
:103CD000DF9300D000D0CDB7DEB78091120690916F
:103CE0001306019709F01CC18091250690912606C4
:103CF000892BD9F40FE110E024E230E04AE550E0EE
:103D000064E670E088E090E00E94A40424E230E0E1
:103D10004AE550E064E670E08FED90E00E94A40474
:103D2000A895A49AAC980E94EB07CC24C394D12CFC
:103D30008091120690911306019709F0F1C0A895A1
:103D400095DE80917506909176068A35910549F445
:103D50002FEF8DE399E4215080409040E1F700C0BF
:103D60000000A89503E02FE130E04FEF5FEF69E13D
:103D700070E085E890E00E94EA1080916300A895C9
:103D80001C821B821A821982BE016F5F7F4FCE0197
:103D900003960E94923D8B819C818431954088F4EA
:103DA00089819A81883D9E4060F489819A81853C11
:103DB000994038F0D0922606C09225061092370618
:103DC000FDD38B819C818431954008F03FC089816F
:103DD0009A818C3D9540D0F589819A81853F9140AB
:103DE000A8F1D0922606C09225061092490680912D
:103DF000140690911506892B11F40E94CD2F809105
:103E0000140690911506019711F40E948D38809147
:103E1000140690911506029711F40E94943980912E
:103E2000140690911506049711F40E94993A809116
:103E3000140690911506059709F448D5809114064B
:103E400090911506069711F40E94C52E8B819C81D6
:103E5000853C994038F089819A818C3D954010F4D9
:103E600089819A81B1DD0E94D20EA8958FEF91EEE3
:103E700024E0815090402040E1F700C00000CDDDFB
:103E8000A8950E94580FE0902D06F0902E0603E0B2
:103E90002FE130E04FEF5FEF6EE670E08CE190E0F5
:103EA0000E94DF05E0907F06F09080062FE130E071
:103EB0004FEF5FEF6EE670E080EF90E00E94DF056D
:103EC0000E94B5108091120690911306892B09F07B
:103ED0002FCFA8950E94FE11A8950E9471110E94F3
:103EE000EB070FE110E024E230E04AE550E064E641
:103EF00070E088E090E00E94A40424E230E04AE50B
:103F000050E064E670E08FED90E00E94A40410920F
:103F1000E6051092E505109226061092250608CFB8
:103F20000F900F900F900F90DF91CF911F910F91F5
:103F3000FF90EF90DF90CF900895EF92FF920F9354
:103F40001F93CF9380913606813009F04BC18FE1EA
:103F500090E00E9419060E94C10B85E080933C0608
:103F6000C5E080913606813009F03CC10E94DD0C2D
:103F700080913C068230D9F4809168068F5F8093EF
:103F800068060FE110E02CE330E046EE50E069E611
:103F900070E081E090E00E94A40422E330E043EC72
:103FA00050E068E270E088E090E00E94A404809114
:103FB0003C068330D9F4809168068150809368066E
:103FC0000FE110E02CE330E046EE50E069E670E0EF
:103FD00081E090E00E94A40422E330E043EC50E052
:103FE00068E270E088E090E00E94A4048091680696
:103FF000853010F01092680680916806823081F159
:10400000B8F48823D9F0813009F0C1C076E8E72EF2
:1040100075E0F72E01E02FE130E04FEF5FEF6CE34A
:1040200070E088E090E00E94990586EB92E029C05C
:104030008330B1F1843009F471C0A9C0EFE9EE2EEC
:10404000E5E0FE2E01E02FE130E04FEF5FEF6CE3A3
:1040500070E08FE090E00E94990588EB92E011C03B
:104060006AE7E62E65E0F62E01E02FE130E04FEF43
:104070005FEF6CE370E082E390E00E94990584EBCF
:1040800092E00E9452427C0103E02FE130E04FEFCA
:104090005FEF62E870E080E590E00E94DF0577C0A6
:1040A00042E6E42E45E0F42E01E02FE130E04FEF50
:1040B0005FEF6CE370E088E290E00E94990550E7C2
:1040C000E52E55E0F52E02E02FE130E04FEF5FEFF7
:1040D00062E870E088E290E00E94990580913C06D9
:1040E000811119C0E3D84FDC3CE2E32E35E0F32E1A
:1040F0002FE130E04FEF5FEF62E870E088E290E0A0
:104100000E9499052FEF89E698E121508040904068
:10411000E1F700C00000C0933C0639C021E5E22E63
:1041200025E0F22E01E02FE130E04FEF5FEF6CE38E
:1041300070E08EE190E00E94990583EB92E00E948E
:104140004A42813079F493E4E92E95E0F92E03E0B8
:104150002FE130E04FEF5FEF62E870E080E590E044
:104160000E94990583EB92E00E944A4281110FC0A0
:104170008EE3E82E85E0F82E03E02FE130E04FEFEC
:104180005FEF62E870E080E590E00E949905809121
:104190003C06813089F41092360610922606109261
:1041A00025068FE190E00E94190681E090E090934F
:1041B00013068093120685DD80913C06811106C0AE
:1041C00081E08093360610927A0612D0C0933C06A6
:1041D0002FE785EB91E0215080409040E1F700C04F
:1041E0000000BFCECF911F910F91FF90EF900895E7
:1041F000BF92CF92DF92EF92FF920F931F93CF93D4
:10420000DF9380917A068111CFC185E080933C06CF
:10421000C9E1D0E025E0C22ED12C35E0B32E80914B
:104220007A068111C1C180916806813009F46FC09E
:1042300038F0823009F4DDC0843009F441C1A4C1F2
:1042400088EB92E00E9452427C0103E02FE130E0D3
:1042500040E058EF62E870E080E590E00E94DF0502
:1042600088EB92E00E94524290933B0680933A067C
:104270000E94DD0C80913C068230A9F480913A06C0
:1042800090913B06019690933B0680933A060FE18E
:1042900010E02CE330E046EE50E069E670E081E0AB
:1042A00090E00E94A40480913C068330A9F48091A0
:1042B0003A0690913B06019790933B0680933A060D
:1042C0000FE110E02CE330E046EE50E069E670E0EC
:1042D00081E090E00E94A40480913A0690913B0610
:1042E0004A9720F0D0933B06C0933A0680913A0655
:1042F00090913B060A9720F4D0933B06C0933A0670
:1043000060913A0670913B0688EB92E066C086EBBE
:1043100092E00E9452427C0103E02FE130E040E055
:1043200058EF62E870E080E590E00E94DF0586EBE0
:1043300092E00E94524290931806809317060E94C2
:10434000DD0C80913C068230A9F480911706909193
:104350001806019690931806809317060FE110E057
:104360002CE330E046EE50E069E670E081E090E05A
:104370000E94A40480913C068330A9F48091170622
:1043800090911806019790931806809317060FE1F5
:1043900010E02CE330E046EE50E069E670E081E0AA
:1043A00090E00E94A40480911706909118064A9705
:1043B00020F0D0931806C0931706809117069091AD
:1043C00018060A9720F4D0931806C0931706609138
:1043D00017067091180686EB92E00E946D422FE757
:1043E00088E391E0215080409040E1F700C0000058
:1043F000CBC084EB92E00E9452427C0103E02FE1AB
:1044000030E040E058EF62E870E080E590E00E9424
:10441000DF0584EB92E00E9452429093390680932C
:1044200038060E94DD0C80913C068230A9F4809110
:104430003806909139060196909339068093380694
:104440000FE110E02CE330E046EE50E069E670E06A
:1044500081E090E00E94A40480913C068330A9F49E
:104460008091380690913906019790933906809390
:1044700038060FE110E02CE330E046EE50E069E64C
:1044800070E081E090E00E94A40480913806909151
:1044900039064F9720F0D0923906C09238068091A5
:1044A000380690913906059720F4D0923906C092CB
:1044B0003806609138067091390684EB92E08DCF12
:1044C00083EB92E00E944A428093DB050E94DD0C60
:1044D00080913C06823089F48091DB058F5F809368
:1044E000DB050FE110E02CE330E046EE50E069E63A
:1044F00070E081E090E00E94A40480913C0683304B
:1045000089F48091DB0581508093DB050FE110E099
:104510002CE330E046EE50E069E670E081E090E0A8
:104520000E94A4048091DB05823010F01092DB051C
:104530008091DB05813079F493E4E92E95E0F92E42
:1045400003E02FE130E040E058EF62E870E080E502
:1045500090E00E9499058091DB0581110FC08EE3E8
:10456000E82E85E0F82E03E02FE130E040E058EF40
:1045700062E870E080E590E00E9499056091DB05BB
:1045800083EB92E00E94604280913C06813049F4C6
:1045900080937A06809336068FE190E00E94190698
:1045A000CCDCB0923C063BCEDF91CF911F910F91B6
:1045B000FF90EF90DF90CF90BF9008954F925F9261
:1045C0006F927F928F929F92AF92BF92CF92DF9223
:1045D000EF92FF920F931F93CF93DF938091370653
:1045E000811163C18FE190E00E9419060E94330B94
:1045F00085E080933C0610923606109230065524D2
:104600005394C7E0D0E0A6E0CA2ED12CB5E0AB2E83
:10461000B12C14E0812E912C03E0602E712C85E0EA
:10462000482E80913706811140C10E94DD0C809197
:104630003C06823089F4809130068F5F809330068B
:104640000FE110E02CE330E046EE50E069E670E068
:1046500081E090E00E94A40480913C06833089F4BC
:10466000809130068150809330060FE110E02CE3FA
:1046700030E046EE50E069E670E081E090E00E94B4
:10468000A40480913006893010F010923006E09139
:1046900030068E2F90E08930910508F0D4C0FC01DF
:1046A000E259FF4F0C942F3FFEE0EF2EF5E0FF2E76
:1046B00002E02FE130E04FEF5FEF62E870E088E06A
:1046C00090E00E94990510923606109215061092FD
:1046D0001406B9C0E0E0EE2EE5E0FE2E02E02FE188
:1046E00030E04FEF5FEF68E770E088E090E00E9415
:1046F00099051092360681E090E013C072EFE72E24
:1047000074E0F72E02E02FE130E04FEF5FEF68E753
:1047100070E088E090E00E9499051092360682E0F1
:1047200090E090931506809314068DC066EEE62EF9
:1047300064E0F62E02E02FE130E04FEF5FEF68E734
:1047400070E088E090E00E94990510923606709221
:1047500015066092140677C054EDE52E54E0F52E50
:1047600002E02FE130E04FEF5FEF68E770E088E0B4
:1047700090E00E949905109236069092150680925C
:10478000140661C03EECE32E34E0F32E02E02FE18C
:1047900030E04FEF5FEF6EE670E088E290E00E945D
:1047A000990544ECE42E44E0F42E2FE130E04FEF85
:1047B0005FEF67E870E08FE090E00E94990510924B
:1047C0003606B0921506A09214063DC027EBE22EE5
:1047D00024E0F22E02E02FE130E04FEF5FEF68E7D8
:1047E00070E088E090E00E94990510923606D09221
:1047F0001506C092140627C099E9E92E94E0F92E17
:1048000002E02FE130E04FEF5FEF68E770E088E013
:1048100090E00E94990510923606D0931506C09339
:10482000140611C083EAE82E84E0F82E02E02FE19E
:1048300030E04FEF5FEF68E770E082E090E00E94C9
:1048400099055092360680913C06813011F5809191
:104850003606813059F41092150610921406109203
:1048600037068FE190E00E94190667DB5092370609
:104870001092260610922506809114069091150636
:1048800090930206809301068FE190E00E94190642
:1048900018DA40923C062FEF80E792E021508040EA
:1048A0009040E1F700C00000BCCEDF91CF911F9196
:1048B0000F91FF90EF90DF90CF90BF90AF909F90BF
:1048C0008F907F906F905F904F900895EF92FF923E
:1048D0000F931F93CF93DF93A89580914906811181
:1048E000F4C08FE190E00E9419060E944F0C809165
:1048F000720690E09093200680931F0685E08093D7
:104900003C06C1E0D5E0809149068111DEC0A89542
:104910000E94DD0C80913C068230A9F480911F0634
:104920009091200601969093200680931F060FE138
:1049300010E02CE330E046EE50E069E670E081E004
:1049400090E00E94A40480913C068330A9F48091F9
:104950001F069091200601979093200680931F06D2
:104960000FE110E02CE330E046EE50E069E670E045
:1049700081E090E00E94A40480911F06909120069F
:10498000039720F01092200610921F0680911F06B8
:10499000909120068130910589F1D0F0029709F0BD
:1049A00046C081E7E82E84E0F82E02E02FE130E0F7
:1049B0004FEF5FEF6DE770E088E290E00E949905AD
:1049C00082E0809372064EE150E06AE570E02BC011
:1049D00025E8E22E24E0F22E02E02FE130E04FEF56
:1049E0005FEF6DE770E088E290E00E949905109219
:1049F00072064EE150E066E970E015C09BE7E92ED3
:104A000094E0F92E02E02FE130E04FEF5FEF6DE729
:104A100070E088E290E00E949905C09372064EE132
:104A200050E068E770E08BEE95E00E943A4280919A
:104A30003C0681110FC0A895C09349061092260626
:104A400010922506C09337068FE190E00E94190668
:104A5000A89537D980913C06813059F5A895809367
:104A600049061092260610922506809337068FE19C
:104A700090E00E941906A895109281068091720616
:104A8000813069F038F0823091F44EE150E06AE50F
:104A900070E009C04EE150E066E970E004C04EE10C
:104AA00050E068E770E08BEE95E00E943A42A895EE
:104AB00013D0D0933C062FEF80E792E02150804046
:104AC0009040E1F700C000001ECFDF91CF911F9111
:104AD0000F91FF90EF900895EF92FF920F931F9325
:104AE000CF938091810681110C94BF2E8FE190E0CD
:104AF0000E9419060E94450D85E080933C06C5E0A2
:104B00008091810681110C94BF2E0E94DD0C809152
:104B10003C068230D9F480916D068F5F80936D06DC
:104B20000FE110E02CE330E046EE50E069E670E083
:104B300081E090E00E94A40422E330E043EC50E0E6
:104B400068E270E088E090E00E94A40480913C0656
:104B50008330D9F480916D06815080936D060FE10A
:104B600010E02CE330E046EE50E069E670E081E0D2
:104B700090E00E94A40422E330E043EC50E068E2BD
:104B800070E088E090E00E94A40480916D068E3071
:104B900010F010926D06E0916D068E2F90E08E3031
:104BA000910508F097C7FC01E958FF4F8091140662
:104BB000909115060C942F3F892B61F57BE2E72E2F
:104BC00074E0F72E01E02FE130E04FEF5FEF62E39A
:104BD00070E08FE090E00E949905E4E2EE2EE4E0C0
:104BE000FE2E2FE130E04FEF5FEF66E470E08CE3E4
:104BF00090E00E949905E090EB05F090EC0503E051
:104C00002FE130E04FEF5FEF62E870E080E590E089
:104C10000E94DF058091140690911506019709F016
:104C20007BC65BE2E52E54E0F52E01E02FE130E09B
:104C30004FEF5FEF62E370E08FE090E00E94990534
:104C400064E2E62E64E0F62E2FE130E04FEF5FEFF6
:104C500066E470E08CE390E00E949905E090EB053B
:104C6000F090EC054EC6892B61F53CE0E32E34E074
:104C7000F32E01E02FE130E04FEF5FEF62E370E0F1
:104C80008FE090E00E9499054EEFE42E43E0F42E71
:104C90002FE130E04FEF5FEF66E470E08CE390E0EF
:104CA0000E949905E090ED05F090EE0503E02FE1FC
:104CB00030E04FEF5FEF62E870E080E590E00E9447
:104CC000DF0580911406909115068130910531F42D
:104CD00080916D068F5F80936D062EC0029761F5FF
:104CE0009CE0E92E94E0F92E01E02FE130E04FEF57
:104CF0005FEF62E370E08FE090E00E9499052EEF95
:104D0000E22E23E0F22E2FE130E04FEF5FEF66E47A
:104D100070E08CE390E00E949905E090ED05F09042
:104D2000EE0503E02FE130E04FEF5FEF62E870E067
:104D300080E590E00E94DF058091140690911506B1
:104D4000049761F50CE0E02E04E0F02E01E02FE185
:104D500030E04FEF5FEF62E370E08FE090E00E94A1
:104D600099058EEFE82E83E0F82E2FE130E04FEF2B
:104D70005FEF66E470E08CE390E00E949905E090BC
:104D8000ED05F090EE0503E02FE130E04FEF5FEF2F
:104D900062E870E080E590E00E94DF0580911406F3
:104DA00090911506059761F5BCE0EB2EB4E0FB2E63
:104DB00001E02FE130E04FEF5FEF62E370E08FE062
:104DC00090E00E9499051EEFE12E13E0F12E2FE1F5
:104DD00030E04FEF5FEF66E470E08CE390E00E941C
:104DE0009905E090ED05F090EE0503E02FE130E04D
:104DF0004FEF5FEF62E870E080E590E00E94DF0532
:104E00008091140690911506069709F063C6FCE0A0
:104E1000EF2EF4E0FF2E01E02FE130E04FEF5FEFE7
:104E200062E370E08FE090E00E949905AEEFEA2E19
:104E3000A3E0FA2E2FE130E04FEF5FEF66E470E081
:104E40008CE390E00E949905E090ED05F090EE056E
:104E5000D8C4892B61F576EEE72E73E0F72E01E0DA
:104E60002FE130E04FEF5FEF62E370E08FE090E022
:104E70000E949905EEECEE2EE3E0FE2E2FE130E0ED
:104E80004FEF5FEF66E470E08FE090E00E949905DD
:104E9000E090EF05F090F00503E02FE130E04FEFF8
:104EA0005FEF62E870E080E590E00E94DF058091AE
:104EB000140690911506019709F02EC556EEE52EC1
:104EC00053E0F52E01E02FE130E04FEF5FEF62E3BA
:104ED00070E08FE090E00E9499056EECE62E63E0B2
:104EE000F62E2FE130E04FEF5FEF66E470E08FE0E9
:104EF00090E00E949905E090EF05F090F00501C563
:104F0000892B61F536EBE32E33E0F32E01E02FE140
:104F100030E04FEF5FEF62E370E08FE090E00E94DF
:104F200099054EE9E42E43E0F42E2FE130E04FEFF7
:104F30005FEF66E470E08FE090E00E949905E090FA
:104F4000F105F090F20503E02FE130E04FEF5FEF65
:104F500062E870E080E590E00E94DF058091140631
:104F6000909115068130910531F480916D068F5F27
:104F700080936D062EC0029761F596EBE92E93E0C3
:104F8000F92E01E02FE130E04FEF5FEF62E370E0D8
:104F90008FE090E00E9499052EE9E22E23E0F22EA8
:104FA0002FE130E04FEF5FEF66E470E08FE090E0DC
:104FB0000E949905E090F105F090F20503E02FE1E1
:104FC00030E04FEF5FEF62E870E080E590E00E9434
:104FD000DF058091140690911506049761F506EBA4
:104FE000E02E03E0F02E01E02FE130E04FEF5FEF25
:104FF00062E370E08FE090E00E9499058EE9E82E70
:1050000083E0F82E2FE130E04FEF5FEF66E470E0D1
:105010008FE090E00E949905E090F105F090F20594
:1050200003E02FE130E04FEF5FEF62E870E080E5F2
:1050300090E00E94DF058091140690911506059777
:1050400061F5B6EBEB2EB3E0FB2E01E02FE130E093
:105050004FEF5FEF62E370E08FE090E00E94990510
:105060001EE9E12E13E0F12E2FE130E04FEF5FEF6C
:1050700066E470E08FE090E00E949905E090F10511
:10508000F090F20503E02FE130E04FEF5FEF62E8D0
:1050900070E080E590E00E94DF0580911406909119
:1050A0001506069709F016C5F6EBEF2EF3E0FF2E76
:1050B00001E02FE130E04FEF5FEF62E370E08FE05F
:1050C00090E00E949905AEE9EA2EA3E0FA2E2FE1C6
:1050D00030E04FEF5FEF66E470E08FE090E00E9419
:1050E0009905E090F105F090F2058BC3892BC9F585
:1050F000E6E8EE2EE3E0FE2E01E02FE130E04FEF98
:105100005FEF6CE370E08FE090E00E949905809182
:10511000F3059091F405019779F473E4E72E75E0B7
:10512000F72E03E02FE130E04FEF5FEF62E870E031
:1051300080E590E00E9499058091F3059091F40537
:10514000892B79F46EE3E62E65E0F62E03E02FE17D
:1051500030E04FEF5FEF62E870E080E590E00E94A2
:10516000990580911406909115060197C9F556E8A6
:10517000E52E53E0F52E01E02FE130E04FEF5FEF39
:105180006CE370E08FE090E00E9499058091F30558
:105190009091F405019779F443E4E42E45E0F42E70
:1051A00003E02FE130E04FEF5FEF62E870E080E571
:1051B00090E00E9499058091F3059091F405892B68
:1051C00079F43EE3E32E35E0F32E03E02FE130E007
:1051D0004FEF5FEF62E870E080E590E00E94990594
:1051E00080911406909115060297C9F526E8E22EE3
:1051F00023E0F22E01E02FE130E04FEF5FEF6CE3B0
:1052000070E08FE090E00E9499058091F305909105
:10521000F405019779F493E4E92E95E0F92E03E083
:105220002FE130E04FEF5FEF62E870E080E590E063
:105230000E9499058091F3059091F405892B79F4EA
:105240008EE3E82E85E0F82E03E02FE130E04FEF0B
:105250005FEF62E870E080E590E00E949905809140
:105260001406909115069C01245031092230310515
:1052700008F4F6C3069709F02DC406E8E02E03E013
:10528000F02E01E02FE130E04FEF5FEF6CE370E0D4
:105290008FE090E00E9499058091F3059091F405CC
:1052A000019779F413E4E12E15E0F12E03E02FE1EC
:1052B00030E04FEF5FEF62E870E080E590E00E9441
:1052C00099058091F3059091F405892B09F002C4AA
:1052D000BEE3EB2EB5E0FB2E03E02FE130E04FEF15
:1052E0005FEF62E870E080E590E00E949905F2C30C
:1052F000892B61F5FEE6EF2EF3E0FF2E01E02FE1B2
:1053000030E04FEF5FEF62E370E08FE090E00E94EB
:105310009905A6E5EA2EA3E0FA2E2FE130E04FEF43
:105320005FEF66E470E08FE090E00E949905E09006
:10533000F505F090F60503E02FE130E04FEF5FEF69
:1053400062E870E080E590E00E94DF05809114063D
:1053500090911506019761F57EE6E72E73E0F72E32
:1053600001E02FE130E04FEF5FEF62E370E08FE0AC
:1053700090E00E949905E6E5EE2EE3E0FE2E2FE197
:1053800030E04FEF5FEF66E470E08FE090E00E9466
:105390009905E090F505F090F60503E02FE130E087
:1053A0004FEF5FEF62E870E080E590E00E94DF057C
:1053B0008091140690911506029761F55EE6E52E40
:1053C00053E0F52E01E02FE130E04FEF5FEF62E3B5
:1053D00070E08FE090E00E94990566E5E62E63E0BC
:1053E000F62E2FE130E04FEF5FEF66E470E08FE0E4
:1053F00090E00E949905E090F505F090F60503E035
:105400002FE130E04FEF5FEF62E870E080E590E081
:105410000E94DF0580911406909115069C0124508E
:1054200031092230310508F41BC3069709F052C335
:105430003EE6E32E33E0F32E01E02FE130E04FEFC4
:105440005FEF62E370E08FE090E00E94990546E52F
:10545000E42E43E0F42E2FE130E04FEF5FEF66E4FF
:1054600070E08FE090E00E949905E090F505F090E3
:10547000F605C7C1892B61F59EE3E92E93E0F92E6D
:1054800001E02FE130E04FEF5FEF62E370E08FE08B
:1054900090E00E94990526E2E22E23E0F22E2FE111
:1054A00030E04FEF5FEF66E470E08FE090E00E9445
:1054B0009905E090F705F090F80503E02FE130E062
:1054C0004FEF5FEF62E870E080E590E00E94DF055B
:1054D0008091140690911506019761F50EE3E02E78
:1054E00003E0F02E01E02FE130E04FEF5FEF62E3E9
:1054F00070E08FE090E00E94990586E2E82E83E05C
:10550000F82E2FE130E04FEF5FEF66E470E08FE0C0
:1055100090E00E949905E090F705F090F80503E00F
:105520002FE130E04FEF5FEF62E870E080E590E060
:105530000E94DF0580911406909115068230910536
:1055400031F480916D068F5F80936D062EC00497B5
:1055500061F5BEE3EB2EB3E0FB2E01E02FE130E07E
:105560004FEF5FEF62E370E08FE090E00E949905FB
:1055700016E2E12E13E0F12E2FE130E04FEF5FEF66
:1055800066E470E08FE090E00E949905E090F705F6
:10559000F090F80503E02FE130E04FEF5FEF62E8B5
:1055A00070E080E590E00E94DF0580911406909104
:1055B0001506059761F5FEE3EF2EF3E0FF2E01E0FF
:1055C0002FE130E04FEF5FEF62E370E08FE090E0BB
:1055D0000E949905A6E2EA2EA3E0FA2E2FE130E020
:1055E0004FEF5FEF66E470E08FE090E00E94990576
:1055F000E090F705F090F80503E02FE130E04FEF81
:105600005FEF62E870E080E590E00E94DF05809146
:1056100014069091150622C2892B61F57EE0E72ED3
:1056200073E0F72E01E02FE130E04FEF5FEF62E330
:1056300070E08FE090E00E949905E6EFEE2EE2E048
:10564000FE2E2FE130E04FEF5FEF66E470E08FE079
:1056500090E00E949905E090F905F090FA0503E0CA
:105660002FE130E04FEF5FEF62E870E080E590E01F
:105670000E94DF05809114069091150681309105F6
:1056800031F480916D068F5F80936D062EC0029776
:1056900061F55EE0E52E53E0F52E01E02FE130E00C
:1056A0004FEF5FEF62E370E08FE090E00E949905BA
:1056B00066EFE62E62E0F62E2FE130E04FEF5FEF6F
:1056C00066E470E08FE090E00E949905E090F905B3
:1056D000F090FA0503E02FE130E04FEF5FEF62E872
:1056E00070E080E590E00E94DF05809114069091C3
:1056F0001506049761F53EE0E32E33E0F32E01E05A
:105700002FE130E04FEF5FEF62E370E08FE090E079
:105710000E94990546EFE42E42E0F42E2FE130E09E
:105720004FEF5FEF66E470E08FE090E00E94990534
:10573000E090F905F090FA0503E02FE130E04FEF3B
:105740005FEF62E870E080E590E00E94DF05809105
:10575000140690911506059761F59EE0E92E93E0F9
:10576000F92E01E02FE130E04FEF5FEF62E370E0F0
:105770008FE090E00E94990526EFE22E22E0F22EC3
:105780002FE130E04FEF5FEF66E470E08FE090E0F4
:105790000E949905E090F905F090FA0503E02FE1E9
:1057A00030E04FEF5FEF62E870E080E590E00E944C
:1057B000DF058091140690911506069709F08AC1BD
:1057C0001EE0E12E13E0F12E01E02FE130E04FEF7B
:1057D0005FEF62E370E08FE090E00E94990586EF52
:1057E000E82E82E0F82E2FE130E04FEF5FEF66E425
:1057F00070E08FE090E00E949905E090F905F0904C
:10580000FA0503E02FE130E04FEF5FEF62E870E070
:1058100080E590E00E94DF055DC1892BF1F4B6E7D9
:10582000EB2EB2E0FB2E01E02FE130E04FEF5FEF17
:105830006CE370E08FE090E00E949905E090030631
:10584000F090040603E02FE130E04FEF5FEF62E8F5
:1058500070E080E590E00E94DF0580911406909151
:105860001506019709F058C0A6E7EA2EA2E0FA2E25
:1058700001E02FE130E04FEF5FEF6CE370E08FE08D
:1058800090E00E949905E0900306F090040639C06C
:10589000892BF1F4FCECEF2EF2E0FF2E01E02FE17A
:1058A00030E04FEF5FEF6CE370E08FE090E00E943C
:1058B0009905E0900506F090060603E02FE130E040
:1058C0004FEF5FEF62E870E080E590E00E94DF0557
:1058D00080911406909115060197F1F4ECECEE2EF0
:1058E000E2E0FE2E01E02FE130E04FEF5FEF6CE3EE
:1058F00070E08FE090E00E949905E0900506F0903E
:10590000060603E02FE130E04FEF5FEF62E870E062
:1059100080E590E00E94DF058091140690911506C5
:105920008230910509F49CC09C0124503109223039
:10593000310508F093C094C0892B09F07CC074EE47
:10594000E72E72E0F72E01E02FE130E04FEF5FEF3E
:105950006CE370E08EE190E00E9499058091FB0578
:105960009091FC05019779F463E4E62E65E0F62E4C
:1059700003E02FE130E04FEF5FEF62E870E080E599
:1059800090E00E9499058091FB059091FC05892B80
:1059900079F45EE3E52E55E0F52E03E02FE130E0EB
:1059A0004FEF5FEF62E870E080E590E00E949905BC
:1059B0008091FB058093DA053EC0892BE1F580914B
:1059C000DA0581110AC010926D0643C0892B99F542
:1059D0008091DA058111AEC1F6CF8130D1F53EE676
:1059E000E32E33E0F32E01E02FE130E04FEF5FEFE5
:1059F00062E370E08FE090E00E94990546EBE42EB0
:105A000042E0F42E2FE130E04FEF5FEF66E470E00C
:105A10008FE090E00E949905E090FD05F090FE0572
:105A200003E02FE130E04FEF5FEF62E870E080E5E8
:105A300090E00E94DF058091140690911506813058
:105A4000910571F08230910559F08430910541F053
:105A500002C080E090E08530910511F00697D1F505
:105A600080916D068F5F80936D0634C0009731F092
:105A70009C01215031092230310518F410926D0635
:105A800020C00497F1F48FE4E82E82E0F82E01E0C4
:105A90002FE130E04FEF5FEF6CE370E08FE090E0DC
:105AA0000E949905E0900706F090080603E02FE1B8
:105AB00030E04FEF5FEF62E870E080E590E00E9439
:105AC000DF0580911406909115060597029710F452
:105AD00010926D0680913C06813009F00EC18093D2
:105AE0008106109249068091140690911506892B23
:105AF00041F5E0911F06F0912006E830F10508F528
:105B0000EB57FF4F4EE150E00C942F3F64E972E0F9
:105B100014C066E772E011C068E572E00EC06AE387
:105B200072E00BC06CE172E008C06EEF71E005C07E
:105B300060EE71E002C062EC71E08BEE95E00E94D5
:105B4000574280911406909115060197E1F48091D7
:105B50001F06909120068130910569F038F0029778
:105B600091F44EE150E068E671E009C04EE150E08A
:105B700064EA71E004C04EE150E066E871E08BEE4B
:105B800095E00E9457428091140690911506029765
:105B9000E1F480911F06909120068130910569F013
:105BA00038F0029791F44EE150E06EE071E009C0E8
:105BB0004EE150E06AE471E004C04EE150E06CE276
:105BC00071E08BEE95E00E9457428091140690910F
:105BD00015060497E1F480911F069091200681300C
:105BE000910569F038F0029791F44EE150E064EBD2
:105BF00070E009C04EE150E060EF70E004C04EE19B
:105C000050E062ED70E08BEE95E00E94574280918B
:105C10001406909115060597E1F480911F06909166
:105C200020068130910569F038F0029791F44EE139
:105C300050E06AE570E009C04EE150E066E970E0CE
:105C400004C04EE150E068E770E08BEE95E00E9402
:105C5000574280911406909115060697E1F48091C1
:105C60001F06909120068130910569F038F0029767
:105C700091F44EE150E060E070E009C04EE150E088
:105C80006CE370E004C04EE150E06EE170E08BEE3A
:105C900095E00E9457428FE190E00E9419068091A2
:105CA000140690911506892B09F477D1809114067A
:105CB00090911506019711F40E948D388091140679
:105CC00090911506029711F40E9494398091140660
:105CD00090911506049711F40E94993A8091140648
:105CE00090911506059711F40E9466248091140680
:105CF00090911506069709F448D080913C068111D1
:105D00000CC081E08093810610924906109209062A
:105D10008FE190E00E941906E3D2C0933C062FE782
:105D200088E391E0215080409040E1F700C00000FE
:105D30000C948025813009F08CCE9FE9E92E92E009
:105D4000F92E01E02FE130E04FEF5FEF62E370E00A
:105D50008FE090E00E9499052CE8E22E22E0F22EDE
:105D60002FE130E04FEF5FEF66E470E08FE090E00E
:105D70000E949905E090FF05F090000651CECF916A
:105D80001F910F91FF90EF900895EF92FF920F9364
:105D90001F93CF93DF93A895809149068111F6C098
:105DA0008FE190E00E9419060E944F0C80916F06CF
:105DB00090E09093200680931F0685E080933C0638
:105DC000C1E0D5E0809149068111E0C0A8950E940C
:105DD000DD0C80913C068230A9F480911F069091E1
:105DE000200601969093200680931F060FE110E095
:105DF0002CE330E046EE50E069E670E081E090E0B0
:105E00000E94A40480913C068330A9F480911F066F
:105E10009091200601979093200680931F060FE132
:105E200010E02CE330E046EE50E069E670E081E0FF
:105E300090E00E94A40480911F0690912006039791
:105E400020F01092200610921F0680911F0690915C
:105E500020068130910589F1D0F0029709F046C003
:105E600081E7E82E84E0F82E02E02FE130E04FEFEA
:105E70005FEF6DE770E088E290E00E94990582E0B4
:105E800080936F064EE150E060E070E02BC025E8A3
:105E9000E22E24E0F22E02E02FE130E04FEF5FEF40
:105EA0006DE770E088E290E00E94990510926F061D
:105EB0004EE150E06CE370E015C09BE7E92E94E002
:105EC000F92E02E02FE130E04FEF5FEF6DE770E079
:105ED00088E290E00E949905C0936F064EE150E081
:105EE0006EE170E08BEE95E00E943A4280913C06B4
:105EF000811110C0A895C0934906109226061092F1
:105F00002506C09337068FE190E00E941906A895F8
:105F10000E94611E80913C06813061F5A8958093B6
:105F200049061092260610922506809337068FE1C7
:105F300090E00E941906A8951092810680916F0644
:105F4000813069F038F0823091F44EE150E060E049
:105F500070E009C04EE150E06CE370E004C04EE137
:105F600050E06EE170E08BEE95E00E943A42A89519
:105F70000E946C25D0933C062FEF80E792E02150E1
:105F800080409040E1F700C000001CCFDF91CF912E
:105F90001F910F91FF90EF900895AF92BF92CF9213
:105FA000DF92EF92FF920F931F93CF93DF93A89509
:105FB00080914906811189C18FE190E00E94190604
:105FC0000E944F0C8091730690E09093200680937E
:105FD0001F0685E080933C06E7E0DE2EF6E0CF2E3C
:105FE000D5E0A4E0BA2EB3E0AB2EC1E08091490623
:105FF00081116BC1A8950E94DD0C80913C06823016
:10600000A9F480911F069091200601969093200696
:1060100080931F060FE110E02CE330E046EE50E0E5
:1060200069E670E081E090E00E94A40480913C0663
:106030008330A9F480911F069091200601979093D8
:10604000200680931F060FE110E02CE330E046EEBF
:1060500050E069E670E081E090E00E94A404809145
:106060001F0690912006089720F0109220061092AB
:106070001F06E0911F06F0912006E830F10508F0B8
:10608000BEC0E357FF4F0C942F3F74E9E72E74E036
:10609000F72E02E02FE130E04FEF5FEF6DE770E0A9
:1060A00082E390E00E949905109273064EE150E061
:1060B00064E972E09AC06FE8E62E64E0F62E02E032
:1060C0002FE130E04FEF5FEF6DE770E082E390E0AB
:1060D0000E949905C09373064EE150E066E772E0B6
:1060E00084C055E8E52E54E0F52E02E02FE130E0C3
:1060F0004FEF5FEF6DE770E088E290E00E94990556
:1061000082E0809373064EE150E068E572E06DC076
:106110004BE7E42E44E0F42E02E02FE130E04FEFB5
:106120005FEF6DE770E088E290E00E949905A09231
:1061300073064EE150E06AE372E057C031E7E32EA8
:1061400034E0F32E02E02FE130E04FEF5FEF6DE738
:1061500070E088E290E00E949905B092730644E1F5
:1061600050E06CE172E041C027E6E22E24E0F22E1E
:1061700002E02FE130E04FEF5FEF6DE770E088E283
:1061800090E00E949905D09373064EE150E06EEFC7
:1061900071E02BC09DE5E92E94E0F92E02E02FE19D
:1061A00030E04FEF5FEF6DE770E088E290E00E9433
:1061B0009905C09273064EE150E060EE71E015C0A3
:1061C00083E5E82E84E0F82E02E02FE130E04FEF87
:1061D0005FEF6DE770E088E290E00E949905D09251
:1061E00073064EE150E062EC71E08BEE95E00E94A8
:1061F0003A428FE59AEE0197F1F700C000008091D6
:106200003C0681110FC0A895C0934906109226063E
:1062100010922506C09337068FE190E00E94190680
:106220000E94611E80913C06813009F041C0A89512
:106230008093490610922606109225068093370611
:106240008FE190E00E94190610928106E09173069A
:106250008E2F90E08830910540F5FC01EB56FF4F02
:106260004EE150E00C942F3F64E972E014C066E701
:1062700072E011C068E572E00EC06AE372E00BC024
:106280006CE172E008C06EEF71E005C060EE71E095
:1062900002C062EC71E08BEE95E00E943A428FE51D
:1062A0009AEE0197F1F700C00000A8950E946C25B6
:1062B000D0933C06A8959FEF20E782E091502040C4
:1062C0008040E1F700C0000091CEDF91CF911F9197
:1062D0000F91FF90EF90DF90CF90BF90AF90089517
:1062E000BF92CF92DF92EF92FF920F931F93CF93C3
:1062F000DF9380910906811106C78FE190E00E942B
:1063000019060E94450D10926E0685E080933C06AA
:1063100098E5C92E92E0D92ECAE5D0E025E0B22E4C
:10632000809109068111EFC6E0916D068E2F90E0F5
:106330008E30910508F0D6C6FC01E356FF4F0C9451
:106340002F3F1BE2E12E14E0F12E01E02FE130E0BF
:106350004FEF5FEF62E370E08FE090E00E949905FD
:1063600084E2E82E84E0F82E2FE130E04FEF5FEF7B
:1063700066E470E08CE390E00E949905E090EB0504
:10638000F090EC0503E02FE130E040E058EF62E8E8
:1063900070E080E590E00E94DF058091EB05909130
:1063A000EC059093DF058093DE050E94DD0C809163
:1063B0003C068230A9F48091DE059091DF050196BC
:1063C0009093DF058093DE050FE110E02CE330E0D1
:1063D00046EE50E069E670E081E090E00E94A4049F
:1063E00080913C068330A9F48091DE059091DF0511
:1063F00001979093DF058093DE050FE110E02CE319
:1064000030E046EE50E069E670E081E090E00E9406
:10641000A4048091DE059091DF058F35914020F036
:106420001092DF051092DE058091DE059091DF0568
:106430009093EC058093EB054CC6ACE0EA2EA4E00B
:10644000FA2E01E02FE130E04FEF5FEF62E370E002
:106450008FE090E00E949905BEEFEB2EB3E0FB2E9B
:106460002FE130E04FEF5FEF66E470E08CE390E007
:106470000E949905E090ED05F090EE0503E02FE114
:1064800030E040E058EF62E870E080E590E00E9484
:10649000DF058091ED059091EE0590933406809391
:1064A00033060E94DD0C80913C068230A9F4809175
:1064B0003306909134060196909334068093330608
:1064C0000FE110E02CE330E046EE50E069E670E0CA
:1064D00081E090E00E94A40480913C068330A9F4FE
:1064E00080913306909134060197909334068093FF
:1064F00033060FE110E02CE330E046EE50E069E6B1
:1065000070E081E090E00E94A404809133069091B5
:106510003406853F914020F01092340610923306E5
:1065200080913306909134069093EE058093ED05AB
:10653000D0C5E6EEEE2EE3E0FE2E01E02FE130E0E6
:106540004FEF5FEF62E370E08FE090E00E9499050B
:10655000FEECEF2EF3E0FF2E2FE130E04FEF5FEF88
:1065600066E470E08FE090E00E949905E090EF050E
:10657000F090F00503E02FE130E040E058EF62E8F2
:1065800070E080E590E00E94DF058091EF0590913A
:10659000F00590937C0680937B060E94DD0C809131
:1065A0003C068230A9F480917B0690917C0601968E
:1065B00090937C0680937B060FE110E02CE330E0A3
:1065C00046EE50E069E670E081E090E00E94A404AD
:1065D00080913C068330A9F480917B0690917C06E3
:1065E000019790937C0680937B060FE110E02CE3EB
:1065F00030E046EE50E069E670E081E090E00E9415
:10660000A40480917B0690917C064F9730F08FE038
:1066100090E090937C0680937B0680917B0690911E
:106620007C060F9730F48FE090E090937C06809387
:106630007B0680917B0690917C069093F005809379
:10664000EF0547C566EBE62E63E0F62E01E02FE18D
:1066500030E04FEF5FEF62E370E08FE090E00E9488
:1066600099057EE9E72E73E0F72E2FE130E04FEF3A
:106670005FEF66E470E08FE090E00E949905E090A3
:10668000F105F090F20503E02FE130E040E058EF33
:1066900062E870E080E590E00E94DF058091F105FE
:1066A0009091F20590931C0680931B060E94DD0CCE
:1066B00080913C068230A9F480911B0690911C06C3
:1066C000019690931C0680931B060FE110E02CE3CB
:1066D00030E046EE50E069E670E081E090E00E9434
:1066E000A40480913C068330A9F480911B0690910C
:1066F0001C06019790931C0680931B060FE110E087
:106700002CE330E046EE50E069E670E081E090E096
:106710000E94A40480911B0690911C064F9730F0B4
:106720008FE090E090931C0680931B0680911B06DF
:1067300090911C060F9730F48FE090E090931C0628
:1067400080931B0680911B0690911C069093F20586
:106750008093F105BEC456E8E52E53E0F52E01E026
:106760002FE130E04FEF5FEF6CE370E08FE090E0FF
:106770000E9499058091F3059091F405019779F4B1
:1067800043E4E42E45E0F42E03E02FE130E040E066
:1067900058EF62E870E080E590E00E9499058091F2
:1067A000F3059091F405892B79F43EE3E32E35E06F
:1067B000F32E03E02FE130E040E058EF62E870E0B4
:1067C00080E590E00E9499058091F305809348064A
:1067D0000E94DD0C80913C06823089F4809148064D
:1067E0008F5F809348060FE110E02CE330E046EE27
:1067F00050E069E670E081E090E00E94A40480919E
:106800003C06833089F48091480681508093480685
:106810000FE110E02CE330E046EE50E069E670E076
:1068200081E090E00E94A40480914806823010F03C
:10683000109248068091480690E09093F40580936A
:10684000F30547C49EE6E92E93E0F92E01E02FE11F
:1068500030E04FEF5FEF62E370E08FE090E00E9486
:10686000990526E5E22E23E0F22E2FE130E04FEFEE
:106870005FEF66E470E08FE090E00E949905E090A1
:10688000F505F090F60503E020E038EF4FEF5FEFFD
:1068900062E870E080E590E00E94DF058091F505F8
:1068A0009091F60590931A06809319060E94DD0CCC
:1068B00080913C068230A9F48091190690911A06C5
:1068C000019690931A06809319060FE110E02CE3CD
:1068D00030E046EE50E069E670E081E090E00E9432
:1068E000A40480913C068330A9F48091190690910C
:1068F0001A06019790931A06809319060FE110E08B
:106900002CE330E046EE50E069E670E081E090E094
:106910000E94A4048091190690911A068B3F91055C
:1069200020F010921A061092190680911906909183
:106930001A069093F6058093F505CBC31EE3E12E6E
:1069400013E0F12E01E02FE130E04FEF5FEF62E363
:1069500070E08FE090E00E94990586E2E82E83E0E7
:10696000F82E2FE130E04FEF5FEF66E470E08FE04C
:1069700090E00E949905E090F705F090F80503E09B
:106980002FE130E040E058EF62E870E080E590E011
:106990000E94DF058091F7059091F80590932C06F1
:1069A00080932B060E94DD0C80913C068230A9F476
:1069B00080912B0690912C06019690932C06809343
:1069C0002B060FE110E02CE330E046EE50E069E6E4
:1069D00070E081E090E00E94A40480913C06833046
:1069E000A9F480912B0690912C06019790932C0688
:1069F00080932B060FE110E02CE330E046EE50E0F0
:106A000069E670E081E090E00E94A40480912B068A
:106A100090912C068536910520F010922C0610924C
:106A20002B0680912B0690912C069093F80580936D
:106A3000F7054FC3AEE0EA2EA3E0FA2E01E02FE106
:106A400030E04FEF5FEF62E370E08FE090E00E9494
:106A50009905B6EFEB2EB2E0FB2E2FE130E04FEFC1
:106A60005FEF66E470E08FE090E00E949905E090AF
:106A7000F905F090FA0503E02FE130E040E058EF2F
:106A800062E870E080E590E00E94DF058091F90502
:106A90009091FA0590932A06809329060E94DD0CB6
:106AA00080913C068230A9F48091290690912A06B3
:106AB000019690932A06809329060FE110E02CE3BB
:106AC00030E046EE50E069E670E081E090E00E9440
:106AD000A40480913C068330A9F48091290690910A
:106AE0002A06019790932A06809329060FE110E069
:106AF0002CE330E046EE50E069E670E081E090E0A3
:106B00000E94A4048091290690912A068536910559
:106B100020F010922A061092290680912906909161
:106B20002A069093FA058093F905D3C2F6E7EF2E73
:106B3000F2E0FF2E01E02FE130E04FEF5FEF6CE37A
:106B400070E08FE090E00E949905E0900306F090DD
:106B5000040603E02FE130E040E058EF62E870E027
:106B600080E590E00E94DF05809103069091040685
:106B700090936A06809369060E94DD0C80913C0622
:106B80008230A9F48091690690916A0601969093EB
:106B90006A06809369060FE110E02CE330E046EED0
:106BA00050E069E670E081E090E00E94A4048091EA
:106BB0003C068330A9F48091690690916A0601979A
:106BC00090936A06809369060FE110E02CE330E0B1
:106BD00046EE50E069E670E081E090E00E94A40497
:106BE0008091690690916A06893C910520F0D093C6
:106BF0006A06C09369068091690690916A068A3593
:106C0000910520F4D0936A06C093690680916906C5
:106C100090916A0690930406809303065AC2ECECA6
:106C2000EE2EE2E0FE2E01E02FE130E04FEF5FEFCD
:106C30006CE370E08FE090E00E949905E09005061B
:106C4000F090060603E02FE130E040E058EF62E804
:106C500070E080E590E00E94DF058091050690914C
:106C600006069093EA058093E9050E94DD0C809169
:106C70003C068230A9F48091E9059091EA050196DD
:106C80009093EA058093E9050FE110E02CE330E0F2
:106C900046EE50E069E670E081E090E00E94A404D6
:106CA00080913C068330A9F48091E9059091EA0532
:106CB00001979093EA058093E9050FE110E02CE33A
:106CC00030E046EE50E069E670E081E090E00E943E
:106CD000A4048091E9059091EA05C39720F01092F1
:106CE000EA051092E9058091E9059091EA059093F3
:106CF000060680930506EDC174EEE72E72E0F72ECE
:106D000001E02FE130E04FEF5FEF6CE370E08EE1E8
:106D100090E00E9499058091FB059091FC050197F8
:106D200079F463E4E62E65E0F62E03E02FE130E02F
:106D300040E058EF62E870E080E590E00E9499053D
:106D40008091FB059091FC05892B79F45EE3E52E9B
:106D500055E0F52E03E02FE130E040E058EF62E827
:106D600070E080E590E00E9499058091FB0580939A
:106D7000DA050E94DD0C80913C06823089F4809116
:106D8000DA058F5F8093DA050FE110E02CE330E045
:106D900046EE50E069E670E081E090E00E94A404D5
:106DA00080913C06833089F48091DA05815080938C
:106DB000DA050FE110E02CE330E046EE50E069E642
:106DC00070E081E090E00E94A4048091DA058230B6
:106DD00010F01092DA058091DA0590E09093FC05AE
:106DE0008093FB0576C18091DA05811103C0109272
:106DF0006D0678C1813009F075C13EE6E32E33E0BF
:106E0000F32E01E02FE130E04FEF5FEF62E370E03F
:106E10008FE090E00E94990546EBE42E42E0F42ECC
:106E20002FE130E04FEF5FEF66E470E08FE090E03D
:106E30000E949905E090FD05F090FE0503E02FE12A
:106E400030E040E058EF62E870E080E590E00E94BA
:106E5000DF058091FD059091FE0590936C0680936F
:106E60006B060E94DD0C80913C068230A9F4809173
:106E70006B0690916C06019690936C0680936B065E
:106E80000FE110E02CE330E046EE50E069E670E000
:106E900081E090E00E94A40480913C068330A9F434
:106EA00080916B0690916C06019790936C0680938D
:106EB0006B060FE110E02CE330E046EE50E069E6AF
:106EC00070E081E090E00E94A40480916B069091B4
:106ED0006C068B3F910520F010926C0610926B06A9
:106EE00080916B0690916C069093FE058093FD0552
:106EF000F0C08091DA05882309F479CF813009F058
:106F0000F1C09FE9E92E92E0F92E01E02FE130E097
:106F10004FEF5FEF62E370E08FE090E00E94990531
:106F20002CE8E22E22E0F22E2FE130E04FEF5FEF6F
:106F300066E470E08FE090E00E949905E090FF0524
:106F4000F090000603E02FE130E040E058EF62E807
:106F500070E080E590E00E94DF058091FF05909150
:106F6000000690934706809346060E94DD0C8091B0
:106F70003C068230A9F4809146069091470601961E
:106F800090934706809346060FE110E02CE330E033
:106F900046EE50E069E670E081E090E00E94A404D3
:106FA00080913C068330A9F4809146069091470673
:106FB000019790934706809346060FE110E02CE37B
:106FC00030E046EE50E069E670E081E090E00E943B
:106FD000A4048091460690914706C39720F0109232
:106FE0004706109246068091460690914706909378
:106FF00000068093FF056DC08FE4E82E82E0F82E36
:1070000001E02FE130E04FEF5FEF6CE370E08FE0E5
:1070100090E00E949905E0900706F090080603E0D2
:107020002FE130E040E058EF62E870E080E590E06A
:107030000E94DF05809107069091080690930F0645
:1070400080930E060E94DD0C80913C068230A9F4EC
:1070500080910E0690910F06019690930F068093F3
:107060000E060FE110E02CE330E046EE50E069E65A
:1070700070E081E090E00E94A40480913C0683309F
:10708000A9F480910E0690910F06019790930F0638
:1070900080930E060FE110E02CE330E046EE50E066
:1070A00069E670E081E090E00E94A4048091E90527
:1070B0009091EA058935924020F0D0920F06C09257
:1070C0000E0680910E0690910F069093080680930D
:1070D00007068FE798E321E0815090402040E1F7D8
:1070E00000C0000080913C06813051F48093090675
:1070F000109281068FE190E00E9419060E946C2593
:10710000B0923C060DC9DF91CF911F910F91FF9076
:10711000EF90DF90CF90BF900895EF92FF920F9382
:107120001F93CF93DF93A895809149068111F5C0F5
:107130008FE190E00E9419060E944F0C80911D067D
:1071400090E09093200680931F0685E080933C0694
:10715000C1E0D5E0809149068111DFC0A8950E9469
:10716000DD0C80913C068230A9F480911F0690913D
:10717000200601969093200680931F060FE110E0F1
:107180002CE330E046EE50E069E670E081E090E00C
:107190000E94A40480913C068330A9F480911F06CC
:1071A0009091200601979093200680931F060FE18F
:1071B00010E02CE330E046EE50E069E670E081E05C
:1071C00090E00E94A40480911F06909120060397EE
:1071D00020F01092200610921F06A89580911F069D
:1071E000909120068130910589F1D0F0029709F045
:1071F00046C081E7E82E84E0F82E02E02FE130E07F
:107200004FEF5FEF6DE770E088E290E00E94990534
:1072100082E080931D064EE150E068E671E02BC0ED
:1072200025E8E22E24E0F22E02E02FE130E04FEFDD
:107230005FEF6DE770E088E290E00E9499051092A0
:107240001D064EE150E064EA71E015C09BE7E92EAF
:1072500094E0F92E02E02FE130E04FEF5FEF6DE7B1
:1072600070E088E290E00E949905C0931D064EE10F
:1072700050E066E871E08BEE95E00E943A42809122
:107280003C0681110FC0A895C093490610922606AE
:1072900010922506C09337068FE190E00E941906F0
:1072A0000E94611E80913C06813059F5A89580931B
:1072B00049061092260610922506809337068FE124
:1072C00090E00E9419061092810680911D0681307F
:1072D00069F038F0823091F44EE150E068E671E0F8
:1072E00009C04EE150E064EA71E004C04EE150E0B4
:1072F00066E871E08BEE95E00E943A42A8950E9404
:107300006C25D0933C062FEF80E792E0215080401F
:107310009040E1F700C000001DCFDF91CF911F9199
:107320000F91FF90EF900895EF92FF920F931F93AC
:10733000CF93DF93A895809149068111F3C08FE127
:1073400090E00E9419060E944F0C8091240690E064
:107350009093200680931F0685E080933C06C1E051
:10736000D5E0809149068111DDC0A8950E94DD0C11
:1073700080913C068230A9F480911F0690912006EE
:1073800001969093200680931F060FE110E02CE3F6
:1073900030E046EE50E069E670E081E090E00E9467
:1073A000A40480913C068330A9F480911F0690913B
:1073B000200601979093200680931F060FE110E0AE
:1073C0002CE330E046EE50E069E670E081E090E0CA
:1073D0000E94A40480911F0690912006039720F03C
:1073E0001092200610921F0680911F069091200691
:1073F0008130910589F1D0F0029709F045C081E70D
:10740000E82E84E0F82E02E02FE130E04FEF5FEF4E
:107410006DE770E088E290E00E94990582E0809339
:1074200024064EE150E06EE071E02BC025E8E22E2C
:1074300024E0F22E02E02FE130E04FEF5FEF6DE746
:1074400070E088E290E00E949905109224064EE1D7
:1074500050E06AE471E015C09BE7E92E94E0F92E54
:1074600002E02FE130E04FEF5FEF6DE770E088E280
:1074700090E00E949905C09324064EE150E06CE232
:1074800071E08BEE95E0F6D780913C06811110C03B
:10749000A895C09349061092260610922506C0931F
:1074A00037068FE190E00E941906A8950E94611EA0
:1074B00080913C06813051F5A89580934906109241
:1074C000260610922506809337068FE190E00E94F1
:1074D00019061092810680912406813069F038F0F7
:1074E000823089F44EE150E06EE071E009C04EE177
:1074F00050E06AE471E004C04EE150E06CE271E0FB
:107500008BEE95E0B7D7A8950E946C25D0933C06EA
:107510002FEF80E792E0215080409040E1F700C0DB
:1075200000001FCFDF91CF911F910F91FF90EF903F
:107530000895EF92FF920F931F93CF93DF93A89537
:10754000809149068111F4C08FE190E00E941906F4
:107550000E944F0C80917E0690E0909320068093CD
:107560001F0685E080933C06C1E0D5E08091490686
:107570008111DEC0A8950E94DD0C80913C0682300E
:10758000A9F480911F069091200601969093200601
:1075900080931F060FE110E02CE330E046EE50E050
:1075A00069E670E081E090E00E94A40480913C06CE
:1075B0008330A9F480911F06909120060197909343
:1075C000200680931F060FE110E02CE330E046EE2A
:1075D00050E069E670E081E090E00E94A4048091B0
:1075E0001F0690912006039720F01092200610921B
:1075F0001F0680911F06909120068130910589F128
:10760000D0F0029709F045C081E7E82E84E0F82E1B
:1076100002E02FE130E04FEF5FEF6DE770E088E2CE
:1076200090E00E94990582E080937E064EE150E052
:1076300064EB70E02BC025E8E22E24E0F22E02E09D
:107640002FE130E04FEF5FEF6DE770E088E290E010
:107650000E94990510927E064EE150E060EF70E0C6
:1076600015C09BE7E92E94E0F92E02E02FE130E00F
:107670004FEF5FEF6DE770E088E290E00E949905C0
:10768000C0937E064EE150E062ED70E08BEE95E037
:10769000F1D680913C06811110C0A895C09349068F
:1076A0001092260610922506C09337068FE190E0CF
:1076B0000E941906A8950E94611E80913C068130A7
:1076C00059F5A89580934906109226061092250632
:1076D000809337068FE190E00E941906A8951092DA
:1076E000810680917E06813069F038F0823089F41D
:1076F0004EE150E064EB70E009C04EE150E060EF15
:1077000070E004C04EE150E062ED70E08BEE95E079
:10771000B1D6A8950E946C25D0933C062FEF80E748
:1077200092E0215080409040E1F700C000001ECF61
:10773000DF91CF911F910F91FF90EF9008950F93DC
:107740001F938091120690911306892B09F099C01E
:10775000809175069091760683359105A9F581E0B3
:1077600090E090931306809312060E9474130FE129
:1077700010E02CE330E044E650E06BE470E08EE68D
:1077800090E00E94A40424E230E04AE550E064E680
:1077900070E088E090E00E94A40424E230E04AE532
:1077A00050E064E670E088E090E00E94A40424E2E7
:1077B00030E04AE550E064E670E08FED90E00E9432
:1077C000A4040E94611EA8950E94361D0E94951374
:1077D000A89503E02FE130E04FEF5FEF69E170E043
:1077E00085E890E00E94EA100E94E41C0E9482104A
:1077F0008091120690911306019781F5A8950E9439
:1078000074130FE110E02CE330E044E650E06BE449
:1078100070E08EE690E00E94A40424E230E04AE5A5
:1078200050E064E670E088E090E00E94A40424E266
:1078300030E04AE550E064E670E088E090E00E94C5
:10784000A40424E230E04AE550E064E670E08FED05
:1078500090E00E94A4040E94611EA8952FEF81EE83
:1078600094E0215080409040E1F700C000000E9469
:10787000D20E0E940D1D0E94580F1F910F910C9463
:10788000C80F1F910F9108951F920F920FB60F927C
:1078900011248F939F938CB190E090937606809300
:1078A00075069F918F910F900FBE0F901F901895A6
:1078B0001F920F920FB60F9211242F938F939F93C5
:1078C0008091E5059091E6050196883E23E09207B8
:1078D00028F49093E6058093E50504C01092E60530
:1078E0001092E50580911006811105C0109278066E
:1078F000109277060BC0813049F480917706909101
:1079000078060196909378068093770680913106E9
:10791000811105C01092E4051092E3050BC081307F
:1079200049F48091E3059091E40501969093E40574
:107930008093E30580912706811105C01092E80528
:107940001092E7050BC0813049F48091E7059091D2
:10795000E80501969093E8058093E7059F918F9144
:107960002F910F900FBE0F901F9018952FEF89E663
:1079700098E1215080409040E1F700C000008FEF77
:107980008ABB81BB8093610081E084BB88EA8FBDA4
:107990008CE08EBD1DBC1CBC17BC16BC8AE78BBD21
:1079A00082E18ABD19BC18BC10927900109278004F
:1079B00080E187BF10BE87E683BF12BE11BE81E89B
:1079C00080938B0085E080938A001092890010924A
:1079D000880010928100109280001092870010920F
:1079E00086001092850010928400109283001092FD
:1079F00082001BB888E98AB986E0809395001092CE
:107A000090008FE289B98FE181BD8FE081BD77D091
:107A100081E00E94B0038FE190E00E94190681E0AE
:107A200090E090931306809312061092260610920F
:107A3000250610921506109214061092E605109273
:107A4000E50510922E0610922D061092E205109276
:107A500011061092790610920A0680E590E0909344
:107A6000760680937506809164008E7F8093640013
:107A700080916500816080936500809164008860DA
:107A8000809364008091650088608093650078949D
:107A9000A49AAC9A2FEF85EA9EE021508040904056
:107AA000E1F700C00000A895AC9882EB92E0F2D418
:107AB000813079F00E945619A8950E94C31CA895A0
:107AC00061E083EB92E0FCD4A89561E082EB92E068
:107AD000F7D4A8958091120690911306019721F48E
:107AE000A8950E94611EA895A89529DEF2CFC0989E
:107AF000AB9AAF9A8FB9779BFECF8FB1089587E08D
:107B000087BBC09AAB9AAF9A83E58DB91EB880E85F
:107B1000EEDF80E0ECDF80E0EADF8AE18A95F1F7D2
:107B200000C00895EF92FF920F931F93CF93DF93BE
:107B300000D000D0CDB7DEB77C018B01A895AB9A01
:107B4000AF9A1C821B821A82198280EDD0DF80E0FE
:107B5000CEDF8FB190E09C838B838B819C81982FAB
:107B600088279C838B8380E0C2DF2FB18B819C812F
:107B7000822B9C838B838B819C8133E096958795A8
:107B80003A95E1F79C838B8387EC90E00197F1F7BE
:107B900000C0000080E9ABDF80E0A9DF8FB190E09A
:107BA0009A83898389819A81982F88279A838983E8
:107BB00080E09DDF2FB189819A81822B9A8389830E
:107BC00089819A8153E0969587955A95E1F79A8332
:107BD00089838B819C81F7019183808389819A813C
:107BE000F801918380830F900F900F900F90DF9199
:107BF000CF911F910F91FF90EF90089570D088F072
:107C00009F5790F0B92F9927B751A0F0D1F0660F88
:107C1000771F881F991F1AF0BA95C9F712C0B130A3
:107C200081F077D0B1E0089574C0672F782F88274E
:107C3000B85F39F0B93FCCF3869577956795B395E2
:107C4000D9F73EF490958095709561957F4F8F4F51
:107C50009F4F0895E89409C097FB3EF49095809556
:107C6000709561957F4F8F4F9F4F9923A9F0F92F02
:107C700096E9BB279395F695879577956795B79580
:107C8000F111F8CFFAF4BB0F11F460FF1BC06F5F66
:107C90007F4F8F4F9F4F16C0882311F096E911C078
:107CA000772321F09EE8872F762F05C0662371F099
:107CB00096E8862F70E060E02AF09A95660F771FAD
:107CC000881FDAF7880F9695879597F9089557FDDD
:107CD0009058440F551F59F05F3F71F04795880F3A
:107CE00097FB991F61F09F3F79F0879508951216D1
:107CF00013061406551FF2CF4695F1DF08C016167D
:107D000017061806991FF1CF86957105610508942D
:107D10000895E894BB2766277727CB0197F9089544
:107D20000BD078C069D028F06ED018F0952309F0F8
:107D30005AC05FC01124EECFCADFA0F3959FD1F3E4
:107D4000950F50E0551F629FF001729FBB27F00D09
:107D5000B11D639FAA27F00DB11DAA1F649F66275E
:107D6000B00DA11D661F829F2227B00DA11D621FAD
:107D7000739FB00DA11D621F839FA00D611D221F67
:107D8000749F3327A00D611D231F849F600D211D4B
:107D9000822F762F6A2F11249F5750408AF0E1F0EE
:107DA00088234AF0EE0FFF1FBB1F661F771F881F37
:107DB00091505040A9F79E3F510570F014C0AACFD2
:107DC0005F3FECF3983EDCF3869577956795B79522
:107DD000F795E7959F5FC1F7FE2B880F911D96954C
:107DE000879597F9089597F99F6780E870E060E0BC
:107DF00008959FEF80EC089500240A941616170644
:107E000018060906089500240A941216130614068B
:107E100005060895092E0394000C11F4882352F0EE
:107E2000BB0F40F4BF2B11F460FF04C06F5F7F4FA6
:107E30008F4F9F4F0895AA1BBB1B51E107C0AA1F7C
:107E4000BB1FA617B70710F0A61BB70B881F991FFB
:107E50005A95A9F780959095BC01CD010895EE0F34
:107E6000FF1F0024001C0BBE0790F691E02D099423
:107E7000A29FB001B39FC001A39F700D811D11246B
:107E8000911DB29F700D811D1124911D0895BB2776
:107E90004A3031F4992322F4BDE2909581959F4FA9
:107EA00001C0BB27FB015527AA27880F991FAA1FCE
:107EB000A41710F0A41B83955051B9F7A05DAA3305
:107EC00008F0A95DA193009779F7B111B1931192D0
:107ED000CB0126C2CF93DF93CDB7DEB7AE014B5FA8
:107EE0005F4FFA0161917191AF0180918406909189
:107EF000850603D0DF91CF9108952F923F924F9244
:107F00005F926F927F928F929F92AF92BF92CF9229
:107F1000DF92EF92FF920F931F93CF93DF93CDB732
:107F2000DEB72B970FB6F894DEBF0FBECDBF6C0146
:107F30007B018A01FC0117821682838181FFBFC108
:107F4000CE0101963C01F6019381F70193FD8591E5
:107F500093FF81917F01882309F4ADC1853239F403
:107F600093FD859193FF81917F01853221F4B601C4
:107F700090E0E6D1E8CF912C212C312CFFE1F315D4
:107F8000D8F08B3279F038F4803279F08332A1F472
:107F9000232D20611DC08D3261F0803369F4232DC3
:107FA000216016C0832D8260382EE32DE4603E2EC2
:107FB0002AC0F32DF8601DC037FC2DC020ED280F1E
:107FC0002A3040F08E32B9F436FC75C1232D20647E
:107FD000322E19C036FE06C08AE0989E200D11246C
:107FE000922E11C0EAE02E9E200D1124222EF32D98
:107FF000F0623F2E08C08C3621F4832D8068382E25
:1080000002C0883641F4F70193FD859193FF819179
:108010007F018111B3CF982F9F7D9554933028F421
:108020000C5F1F4F9FE399830DC0833631F0833778
:1080300071F0833509F055C020C0F8018081898333
:108040000E5F1F4F88248394912C530112C0280186
:10805000F2E04F0E511CF801A080B18036FE03C043
:10806000692D70E002C06FEF7FEFC5014ED14C016A
:108070008201F32DFF773F2E15C0280122E0420E2A
:10808000511CF801A080B18036FE03C0692D70E05C
:1080900002C06FEF7FEFC5012DD14C01F32DF068C9
:1080A0003F2E820133FC19C0822D90E0881699067C
:1080B000A0F4B60180E290E043D12A94F5CFF50117
:1080C00037FC859137FE81915F01B60190E038D190
:1080D00021102A9421E0821A91088114910479F7E1
:1080E000E1C0843611F0893639F5F80137FE07C052
:1080F00060817181828193810C5F1F4F08C0608114
:108100007181072E000C880B990B0E5F1F4FF32D0A
:10811000FF763F2E97FF09C09095809570956195E9
:108120007F4F8F4F9F4FF0683F2E2AE030E0A30132
:1081300043D1882E861844C0853731F4232D2F7EF5
:10814000B22E2AE030E025C0932D997FB92E8F36CC
:10815000C1F018F4883579F0AEC0803719F088374F
:1081600021F0A9C0E92FE061BE2EB4FE0DC0FB2DA9
:10817000F460BF2E09C034FE0AC0292F2660B22E3B
:1081800006C028E030E005C020E130E002C020E178
:1081900032E0F801B7FE07C060817181828193816E
:1081A0000C5F1F4F06C06081718180E090E00E5F20
:1081B0001F4FA30101D1882E8618FB2DFF773F2E7C
:1081C00036FE0DC0232D2E7FA22E891458F434FEC6
:1081D0000BC032FC09C0832D8E7EA82E05C0B82CA2
:1081E000A32C03C0B82C01C0B92CA4FE0FC0FE0103
:1081F000E80DF11D8081803321F49A2D997EA92EFE
:1082000009C0A2FE06C0B394B39404C08A2D867838
:1082100009F0B394A3FC10C0A0FE06C0B21480F411
:10822000280C922C9B180DC0B21458F4B60180E2B1
:1082300090E086D0B394F8CFB21418F42B1802C093
:10824000982C212CA4FE0FC0B60180E390E078D0DA
:10825000A2FE16C0A1FC03C088E790E002C088E53A
:1082600090E0B6010CC08A2D867851F0A1FE02C0C4
:108270008BE201C080E2A7FC8DE2B60190E060D005
:10828000891430F4B60180E390E05AD09A94F8CF84
:108290008A94F301E80DF11D8081B60190E050D081
:1082A0008110F6CF222009F44ECEB60180E290E094
:1082B00047D02A94F7CFF6018681978102C08FEFCD
:1082C0009FEF2B960FB6F894DEBF0FBECDBFDF91A8
:1082D000CF911F910F91FF90EF90DF90CF90BF90C3
:1082E000AF909F908F907F906F905F904F903F9056
:1082F0002F900895FC010590615070400110D8F74F
:10830000809590958E0F9F1F0895FC0161507040DD
:1083100001900110D8F7809590958E0F9F1F0895BA
:10832000DC01FC01672F71917723E1F7329704C0DC
:108330007C916D9370836291AE17BF07C8F3089567
:108340000F931F93CF93DF93FB01238121FD03C084
:108350008FEF9FEF2CC022FF16C0468157812481EA
:1083600035814217530744F4A081B1819D012F5FED
:108370003F4F318320838C93268137812F5F3F4F7E
:108380003783268314C08B01EC01FB010084F18547
:10839000E02D0995892BE1F6D80116968D919C91D7
:1083A0001797019617969C938E931697CE01DF919F
:1083B000CF911F910F910895FA01AA27283051F10A
:1083C000203181F1E8946F936E7F6E5F7F4F8F4F06
:1083D0009F4FAF4FB1E03ED0B4E03CD0670F781F65
:1083E000891F9A1FA11D680F791F8A1F911DA11D4A
:1083F0006A0F711D811D911DA11D20D009F4689483
:108400003F912AE0269F11243019305D3193DEF62A
:10841000CF010895462F4770405D4193B3E00FD0E0
:10842000C9F7F6CF462F4F70405D4A3318F0495DCB
:1084300031FD4052419302D0A9F7EACFB4E0A695AE
:108440009795879577956795BA95C9F700976105D0
:10845000710508959B01AC010A2E06945795479526
:1084600037952795BA95C9F7620F731F841F951F1B
:10847000A01D0895DC01CB01FC01E199FECF06C0EF
:10848000FFBBEEBBE09A31960DB20D9241505040C9
:10849000B8F70895E199FECF9FBB8EBBE09A99276C
:1084A0008DB30895A8E1B0E042E050E0E5CFDC01F3
:1084B000CB0102C02D9105D041505040D8F708950E
:1084C000262FE199FECF9FBB8EBB2DBB0FB6F89434
:1084D000E29AE19A0FBE01960895F2DF272FF1CFBD
:0484E000F894FFCF3E
:1084E4000000000200000000DE07000000005754F6
:1084F4003D2025750A47530047533D2025750A53EF
:108504004E00534E3D2025750A454E4400574B3DC1
:108514002025750A565000503D332E360A5200521B
:108524004C3D2025750A68004F3D73740A5300477B
:108534003D73740A530053523D53746174696F6EF2
:10854400200A57500057503D536E36332F50623334
:10855400370A57540057503D536E41670A57540029
:1085640057503D50726F66696C65300A5754005716
:10857400503D50726F66696C65310A57540057500C
:108584003D50726F66696C65320A57540057503D0E
:1085940050726F66696C65330A57540057503D50EA
:1085A400726F66696C65340A57540057503D5072B7
:1085B4006F66696C65350A57540053523D555068CF
:1085C4006561746572200A57500053523D507265BC
:1085D400686561746572200A57500053523D4D61BD
:1085E4006E75616C200A57500053523D5265626F9C
:1085F4006C6C696E67200A57500053523D4368699A
:108604007068656174696E67200A57500053523D63
:1086140050434268656174696E67200A575000537D
:10862400523D5043200A57500056312E307A0020D4
:108634002020C2F0E5ECFF20F0E5E1EEEBEBE8ED05
:10864400E3E02020202000C2FBE1E5F0E8F2E52091
:10865400F0E5E6E8EC00D2E5ECEFE5F0E0F2F3F06B
:10866400E020EFEEEBEEF7EAE8202000EDE8E7E0AB
:1086740020EFF0E820E4EEEDE0E3F0E5E2E500D2FF
:10868400E5ECEFE5F0E0F2F3F0E020F3E2E5EBE80F
:10869400F7E5EDE8FF00202020202020E4EEEDE0C7
:1086A400E3F0E5E2E020202020202000C4EBE8F203
:1086B400E5EBFCEDEEF1F2FC20E2EFE8F2FBE2E0A8
:1086C400EDE8FF00D4F3EDEAF6E8FF20E4EEEDEE8A
:1086D400E3F0E5E2E000EDE8E6EDE5E3EE20EDE0D1
:1086E400E3F0E5E2E0F2E5EBFF2020202000CCE01F
:1086F400EAF1E8ECE0EBFCEDE0FF20ECEEF9EDEE66
:10870400F1F2FC202000E2E5F0F5EDE5E3EE20EDEA
:10871400E0E3F0E5E2E0F2E5EBFF20202000CCE02E
:10872400EAF1E8ECE0EBFCEDE0FF20ECEEF9EDEE35
:10873400F1F2FC202000E2E5F0F5EDE5E3EE20EDBA
:10874400E0E3F0E5E2E0F2E5EBFF20202000D2E5F3
:10875400ECEFE5F0E0F2F3F0E020E2EAEBFEF7E51F
:10876400EDE8FF202000CAEEEDF2F0EEEBFC20EF86
:10877400EE20E2E5F0F5F320202020202000EDE8B3
:10878400E6EDE5E3EE20EDE0E3F0E5E2E0F2E5EB33
:10879400FF2020202000CAEEFDF4F4E8F6E8E5ED21
:1087A400F220EFF0EEF4E8EBFF2020202000E2E5D9
:1087B400F0F5EDE5E3EE20EDE0E3F0E5E2E0F2E5EF
:1087C400EBFF20202000CAEEFDF4F4E8F6E8E5ED26
:1087D400F220EFF0EEF4E8EBFF2020202000EDE0A3
:1087E400E3F0E5E2E0F2E5EBFF202000D2E5ECEF78
:1087F400E5F0E0F2F3F0E020EDE8E6EDE5E3EE206D
:1088040020202000EFE0E9EAE82000D2E5ECEFE5E3
:10881400F0E0F2F3F0E020ECE5F1F2E0202020209B
:108824002000C2FBE1E5F0E8F2E520EFF0EEF4E829
:10883400EBFC00CFF0EEF4E8EBFC203500CFF0EEDB
:10884400F4E8EBFC203400CFF0EEF4E8EBFC20334A
:1088540000CFF0EEF4E8EBFC203200CFF0EEF4E8C9
:10886400EBFC203100CFF0EEF4E8EBFC20300053B9
:108874006E416700536E506200CAEEECEFFCFEF2EC
:10888400E5F000C4EEEF2E20EDE0F1F2F0EEE9EABF
:10889400E800EFEBE0F20020D1F3F8EAE020EFEBA0
:1088A400E0F22000ECE8EAF0EEF1F5E5EC00D1F3BB
:1088B400F8EAE000D0E5E1EEEBEBE8EDE32000D0F0
:1088C400F3F7EDEEE9002020D0F3F7EDEEE92020F8
:1088D4002000CDE8E6EDE8E920EDE0E3F02E20000D
:1088E400C2E5F0F5EDE8E920EDE0E3F02E0020200C
:1088F400D1F2E0EDF6E8FF00E2E5F0F5E000EDE8A6
:10890400E7E000CCEEF9EDEEF1F2FC00CFF0E8ED9B
:10891400FFF2EE202000C2DBC1D0C0D2DC00C2DBFB
:10892400CACB00C2CACB00CDE0F1F2F0EEE8F2FC13
:1089340000C7E2F3EAEEE2FBE520F1E8E3EDE0EB69
:10894400FB00CFF0E5E4F3F1F2E0EDEEE2EAE8005B
:10895400D3ECEEEBF7E0EDE8FF00C2F0E5ECFF202E
:10896400EFE0E9EAE80020C4E0F2F7E8EA20EDE805
:10897400E62E20EDE0E3F0E5E2E0F2E5EBFF002097
:10898400C4E0F2F7E8EA20ECE5F1F2E020EFE0E9F8
:10899400EAE800F0F3F7EDEEE900EDE8E6EDE8E9EA
:1089A40000EDE0E3F02E00C2E5F0F5EDE8E900C2E9
:0689B400DBD5CEC400007B
:00000001FF
